:1000000002D4A7CFC39FFF50011E22021FE100FCB4
:10001000F8F0E1C2000096004B00258012C0096094
:1000200068A8E802D367A3E004F0700612D48BE05E
:1000300004F02202D38200FCF8F0E1C20000960036
:100040004B00258012C0096068A8E82077616974B8
:100050005F69722000204E6F206465636B207479A5
:1000600070652073656C65637465640D0A005341A7
:100070004E32010000630016001A00180019001823
:100080000019001A003000190030001B0017001A78
:100090000017001B0017001A002F001C0016001C80
:1000A000002D001C002E001C002D001C002E001D29
:1000B0000015001C0015001D002D001D0015001E60
:1000C000002D001D00140215005D001D0014001D10
:1000D0000015001D0014001D002D001D002C001D2A
:1000E0000015001D0014001D0015001E002C001D31
:1000F0000015001D002C001D002C001F002C001EF0
:10010000002C001F0014001D0014001E002C001EF7
:100110000014001E002C001D001402160000000038
:10012000000000000000000000620017001A001824
:10013000003100180018001A0030001A002F001BB0
:100140000017001A0016001B0016001B002F001CD1
:100150000016001C002D001C002E001C002D001C91
:10016000002E001D0015001C0015001D002D001D97
:100170000014001E002C001D001401FC005E001D78
:100180000014001E002C001D0014001D002D001D79
:10019000002C001D0015001D0014001D0014001D82
:1001A000002C001D0015001E002C001D002B001F40
:1001B000002C001E002B001F0014001D0014001E48
:1001C000002C001E0013001E002C001D001401FD59
:1001D00000000000000000000000000000620016A7
:1001E000001A0017001A0018003100190030001919
:1001F0000030001B0017001A0017001B0017001A20
:10020000002F001C0016001B002E001C002E001CDE
:10021000002D001C002E001D0015001C0014001EE7
:10022000002D001C0014001E002D001D001401FCF8
:10023000005E001C0015001C0016001C002D001D97
:10024000002D001D002C001D0015001D0014001DB8
:100250000015001D002C001D0015001D002C001DA8
:10026000002C001F002C001D002B001F0014001D7F
:100270000014001E002C001D0014001E002C001D88
:10028000001401FD0000000000000000000000005C
:100290000062001600320019003100190018001A1F
:1002A000002F001A002F001B0017001A0017001C57
:1002B0000016001B002E001C0016001C002D001C48
:1002C000002E001D002D001C002D001D0014001D1F
:1002D0000014001E002D001D0014001E002D001D26
:1002E000001401E3005E001C002D001D002E001D07
:1002F0000014001D002D001D002D001D0015001D07
:100300000014001D0014001E002C001D0013001F0F
:10031000002C001D002C001E002C001E002B001FB6
:100320000014001D0014001E002C001E0013001EEF
:10033000002C001D001401E400000000000000007B
:1003400000000000006100160032001900190018BA
:100350000018001A003000190030001B0017001AA6
:100360000017001B0017001A002F001C0016001BAE
:10037000002E001C002E001C002D001C002E001D55
:100380000015001C0014001E002D001C0015001E8E
:10039000002D001D001401FC005E001C002D001D3E
:1003A0000015001D0014001D002D001D002D001D56
:1003B0000015001D0014001D0015001D002D001D5E
:1003C0000014001E002C001D002B001F002C001E1E
:1003D000002B001F0014001D0014001E002C001E26
:1003E0000013001F002C001D001401FD0000000080
:1003F000000000000000000000620017003100193A
:10040000001900180031001A0030001A002F001BDC
:100410000017001A0016001C0016001C002D001CFE
:100420000016001C002D001C002E001D002D001CBD
:10043000002D001D0014001D0015001D002C001DC6
:100440000014001E002C001D001401E3005E001DBE
:10045000002C001D0015001D002C001D002D001D8E
:10046000002C001D0015001D0014001D0015001EAD
:10047000002C001D0013001F002C001D002B001F6E
:10048000002C001D002B00200014001D0014001E75
:10049000002C001D0014001E002C001D001401E59E
:1004A00000000000000000000000000000630016D3
:1004B000001A0018003100190031001A0017001A44
:1004C000002F001B0017001A002F001B0016001B36
:1004D000002E001C0016001C002D001C002E001D0C
:1004E000002D001C002E001D0015001C0014001E15
:1004F000002D001D0014001E002D001D001401E33E
:10050000005E001D0014001D002E001D002D001DAA
:100510000015001D002C001D0015001D002C001DE5
:100520000015001E002C001D0013001F002C001DD4
:10053000002C001F002C001D002B001F0014001DAC
:100540000014001E002C001E0013001E002C001DB5
:10055000001401E4000000000000000000000000A2
:100560000062001700320019003000190017001A4D
:100570000030001A002F001B0016001B0015001C85
:100580000016001C002D001C0016001C002D001C75
:10059000002E001D002D001D002D001D0014001D4B
:1005A0000015001D002C001D0014001E002C001D55
:1005B000001401E3005E001D002D001D002D001D34
:1005C0000014001D002D001D002C001D0015001D35
:1005D0000014001D0015001E002C001E0013001E3C
:1005E000002C001D002B001F002C001E002B001FE4
:1005F0000014001D0014001E002C001E0013001E1D
:10060000002C001D001401E40000000000000000A8
:100610000000000000620016001A001800310018E7
:100620000031001A0017001A0030001B0017001AD2
:10063000002F001B0016001B002F001C0016001CC2
:10064000002D001C002E001D002D001C002E001D82
:100650000015001C0014001E002D001D0014001EBB
:10066000002D001D001401E3005E001D0014001D9C
:10067000002E001D002D001D0015001D002D001D69
:100680000015001D002D001D0014001E002C001D73
:100690000013001F002C001D002C001E002C001D4C
:1006A000002B001F0013001E0014001E002C001D54
:1006B0000014001E002C001D001401E300000000C7
:1006C0000000000000000000006100170031001968
:1006D000003100190030001B0017001A002F001B0A
:1006E0000016001C002D001C0016001C002D001C14
:1006F0000016001C002D001C002E001D002D001DEA
:10070000002D001D0014001D0015001E002C001DF2
:100710000014001E002C001D001401CC005D001D03
:10072000002D001E002C001D002C001D0015001DBA
:10073000002C001E0014001E002C001D0015001DC2
:10074000002C001E0013001F002C001D002B001F9A
:10075000002C001E002B001F0014001D0014001EA2
:10076000002C001E0013001E002C001D001401CCE4
:100770000000000000000000000000000063001600
:10078000001A0018001900180031001A001800198A
:100790000017001A0030001A0017001B0017001A7B
:1007A000002F001C0016001C002D001C002E001C39
:1007B000002D001C002E001D0015001C0015001E41
:1007C000002D001D0014001E002D001D0014021538
:1007D000005D001C0015001D0015001D002D001DF2
:1007E0000015001D0014001D002D001D0014001D2B
:1007F0000015001D002D001D0014001E002C001D02
:10080000002B001F002C001E002B001F0014001DD9
:100810000014001E002C001E0013001E002C001DE2
:10082000001402160000000000000000000000009C
:100830000062001600320019003100190018001A79
:10084000003000190017001B0017001A0017001BCA
:100850000017001A002F001C0016001B002E001CA1
:10086000002E001B002E001C002E001C0015001C7A
:100870000015001D002D001C0015001D002D001D81
:10088000001401FC005E001C002D001D002E001D48
:100890000014001D002D001D0014001D0015001D7A
:1008A0000014001D0015001D002C001D0015001D6A
:1008B000002D001D002C001E002C001D002B001F11
:1008C0000013001E0013001E002C001D0014001E4B
:1008D000002C001E001301FD0000000000000000BD
:1008E0000000000000620016001A00170032001815
:1008F00000180019001900190018001A0017001A32
:100900000030001B0017001A002F001B0016001BF0
:10091000002F001C002E001B002E001C002E001CAF
:100920000016001C0015001C002E001C0015001DE8
:10093000002D001C00140214005E001B0016001C99
:10094000002E001C0015001D0015001D0014001DC8
:100950000015001D002D001D0015001D002D001D9F
:100960000013001F002C001D002C001E002D001D78
:10097000002C001E0014001D0014001E002C001D81
:100980000014001E002C001D0014021500000000C1
:100990000000000000000000006200160032001895
:1009A000003200190018001A001800190018001A67
:1009B0000017001A002F001B0017001A002F001C40
:1009C0000016001B002F001C002E001B002E001C18
:1009D000002D001C0016001C0015001D002D001C21
:1009E0000015001D002D001D001401FC005E001C00
:1009F000002D001D002E001D0014001D0015001DFF
:100A00000014001D0015001D002D001D0014001E07
:100A1000002C001D0014001E002D001D002D001EC6
:100A2000002C001D002C001E0013001E0013001ED1
:100A3000002C001D0014001E002C001E001301FDE0
:100A4000000000000000000000000000006300162D
:100A5000001A0018003100180018001A00180019B8
:100A60000018001A0030001A002F001B0017001A8F
:100A7000002F001C0016001B002E001C002E001C66
:100A8000002D001C002D001D0015001C0014001E70
:100A9000002D001D0014001E002D001D001401FC7F
:100AA000005E001C0015001C002E001D0014001D1F
:100AB0000015001D0014001D002D001D002D001D3F
:100AC0000015001E002C001D0015001D002C001D2F
:100AD000002C001E002C001D002B001F0014001D08
:100AE0000014001E002C001E0013001E002C001D10
:100AF000001401FD000000000000000000000000E4
:100B00000062001600320019001900180018001ABF
:100B1000001800190018001A0030001A002F001BDE
:100B20000017001A002F001C0016001B002E001CCE
:100B3000002E001B002E001C002D001D0015001CA7
:100B40000014001E002D001D0014001E002D001DAD
:100B5000001401FC005E001C002D001C0016001D8E
:100B60000014001D0015001D0014001D002D001DA7
:100B7000002D001D0014001E002D001D0014001E7D
:100B8000002C001D002C001E002C001E002B001F3E
:100B90000014001D0014001E002C001E0014001E76
:100BA000002C001D001401FD0000000000000000EA
:100BB0000000000000620016003200180032001928
:100BC0000018001A001800190018001B002F001A46
:100BD0000017001B0017001A002F001B0016001B37
:100BE000002E001C002E001C002E001C002D001CDE
:100BF0000016001C0015001D002D001C0015001D16
:100C0000002D001D001401FC005E001C002D001DC5
:100C1000002E001D0014001D0015001D0014001DF5
:100C2000002D001D0014001D0014001E002C001DCE
:100C30000014001E002D001D002D001E002C001DA4
:100C4000002C001E0013001E0013001E002C001DAF
:100C50000014001E002C001E001301FD0000000007
:100C6000000000000000000000620016001A0017DB
:100C70000032001800180019001900190018001A95
:100C80000031001A0017001A0018001A002F001B6C
:100C90000016001B002E001C002E001B002E001C46
:100CA000002D001C0016001C0015001C002E001C4E
:100CB0000015001D002D001D00140214005E001B15
:100CC0000016001C002E001C0015001D0015001D44
:100CD0000014001D002E001D0014001D0014001E35
:100CE000002D001D0013001F002C001D002C001EF5
:100CF000002C001E002C001E0014001D0014001EFD
:100D0000002C001E0013001E002C001D00140215F4
:100D1000000000000000000000000000006200175A
:100D200000320019001800190018001A0030001ACB
:100D30000017001B0017001A0017001B0017001BEC
:100D4000002E001C0016001C002D001C002E001D93
:100D5000002D001C002D001D0015001C0015001E9C
:100D6000002C001D0014001E002C001D0014021594
:100D7000005D001D002C001D0015001D0014001D4D
:100D8000002D001D0014001D0015001D0014001D85
:100D90000015001D002C001D0014001D002C001D5E
:100DA000002B001F002C001D002B001F0014001D35
:100DB0000014001E002C001D0014001E002C001D3D
:100DC00000140215000000000000000000000000F8
:100DD00000620017001A0018001900180018001A05
:100DE000001800190018001A0017001A0017001B3D
:100DF0000017001A002F001B0016001C002D001CFD
:100E0000002E001C002D001C002E001C0015001CD4
:100E10000015001D002D001D0015001E002D001DD9
:100E200000140246005D001D0014001D0015001D89
:100E30000014001D0015001D0014001D0015001DEC
:100E40000014001D0015001D002C001D0015001EC3
:100E5000002C001D002C001E002C001D002D001E6B
:100E60000014001D0013001F002C001D0014001EA4
:100E7000002C001D001402470000000000000000CC
:100E8000000000000062001600320019001800196E
:100E90000018001A001800190018001A0017001A8C
:100EA0000017001B0017001A002F001B0016001C63
:100EB000002E001C002E001C002D001C002E001D0A
:100EC0000015001C0015001D002D001C0014001E44
:100ED000002C001D0014022D005D001C002D001DC3
:100EE0000015001D0014001D0015001D0014001D3C
:100EF0000015001D0014001D0015001D002D001D13
:100F00000015001E002C001D002B001F002C001DD2
:100F1000002B001F0014001D0014001E002C001DDB
:100F20000014001E002C001D0014022D0000000003
:100F3000000000000000000000620016001A001807
:100F4000003100180018001A001800190018001AC3
:100F50000017001A0017001B0017001A002F001BB3
:100F60000017001B002F001C002E001B002E001C71
:100F7000002E001B0016001C0015001D002D001C7B
:100F80000015001D002D001C0015022C005E001B2A
:100F90000016001C002E001C0015001C0016001C72
:100FA0000015001D0015001D0014001D0015001D7A
:100FB000002D001D0015001D002D001D002C001F20
:100FC000002C001D002D001D0014001D0014001E2B
:100FD000002C001D0014001E002C001D0014022D0A
:100FE0000000000000000000000000000062001689
:100FF00000320019003100190018001A00180019F9
:101000000017001B0017001A0017001B0017001A1A
:10101000002F001B0016001B002F001C002E001BC1
:10102000002E001C002D001D0015001C0015001DC9
:10103000002D001C0014001E002D001D00140215C0
:10104000005D001C002D001C002E001D0014001D62
:101050000015001D0014001D0015001D0014001DCA
:101060000015001D002D001D0014001E002C001D89
:10107000002C001E002C001E002B001F0014001D61
:101080000014001E002C001E0013001E002C001D6A
:101090000014021500000000000000000000000025
:1010A00000620016001A0018001900180031001A1A
:1010B000001800190018001A0017001A0017001B6A
:1010C0000017001A002F001B0017001A002F001C29
:1010D000002E001B002E001C002E001C0015001C02
:1010E0000015001D002D001C0015001D002D001D09
:1010F0000014022C005E001C0015001C0016001CD1
:10110000002D001D0015001D0014001D0015001D00
:101110000014001D0015001D002D001D0015001EEF
:10112000002C001D002C001F002C001D002D001E97
:101130000014001D0014001E002C001D0014001ED1
:10114000002C001D0014022D000000000000000013
:10115000000000000062001600320019001900189B
:101160000031001A001800190017001B0017001AA0
:101170000017001B0017001A002F001C0016001B90
:10118000002E001C002E001C002D001C002D001D38
:101190000015001C0015001D002D001D0014001E70
:1011A000002D001D00140215005D001C002D001C08
:1011B0000016001D002C001D0015001D0014001D50
:1011C0000015001D0014001D0015001D002D001D40
:1011D0000014001E002C001D002C001E002C001D01
:1011E000002B001F0014001D0014001E002C001E08
:1011F0000013001E002C001D00140215000000004A
:10120000000000000000000000620016001A001834
:10121000003100180031001A001800190017001BD7
:101220000017001A0017001B0017001A002F001BE0
:101230000016001B002F001C002E001C002D001C9F
:10124000002E001D0015001C0015001D002D001CA7
:101250000015001E002D001D00140214005E001C6D
:101260000015001D002D001C002D001D0015001D87
:101270000014001D0015001D0014001D0015001DA8
:10128000002C001D0015001D002D001D002B001F4F
:10129000002C001D002D001E0013001E0014001E57
:1012A000002C001D0014001E002C001E001402154E
:1012B00000000000000000000000000000630016B5
:1012C00000320019003100190030001A0017001A0E
:1012D0000017001B0017001A0017001B0017001A48
:1012E000002F001C0016001B002E001C002E001CEE
:1012F000002D001C002D001D0015001C0014001EF8
:10130000002D001D0014001E002D001D001401FC06
:10131000005E001D002D001D002D001D002D001D74
:101320000015001D0014001D0015001D0014001DF7
:101330000014001D002C001D0015001D002C001DB8
:10134000002C001E002C001D002B001F0014001D8F
:101350000014001E002C001D0014001E002C001D97
:10136000001401FD0000000000000000000000006B
:1013700000620016001A0018001900180019001960
:10138000003100190018001A0017001A0017001B7E
:101390000017001A002F001B0017001A002F001C56
:1013A000002E001B002E001C002E001C0015001C2F
:1013B0000015001D002D001C0015001E002D001D35
:1013C0000014022C005E001C0015001C0016001CFE
:1013D0000015001C002E001C0015001D0015001D2E
:1013E0000014001D0015001D002C001D0015001D1F
:1013F000002D001D002C001F002C001D002D001DC5
:101400000014001D0014001E002C001D0014001EFE
:10141000002C001E0013022D000000000000000040
:1014200000000000006200170032001900190019C6
:101430000030001A0017001A0030001B0017001AB5
:101440000017001B0017001B002E001C0016001CBC
:10145000002D001C002E001C002D001C002E001D65
:101460000014001D0015001D002D001D0014001E9D
:10147000002C001D001401FD005D001D002D001D4D
:101480000015001D002D001D0015001D002C001D65
:101490000015001D0014001D0015001E002C001D6D
:1014A0000015001D002C001E002D001E002C001D2C
:1014B000002C001F0013001E0012001F002C001D36
:1014C0000014001E002C001E001301FD000000008F
:1014D000000000000000000000620016001A001862
:1014E000003200180031001A001800190030001BEB
:1014F0000017001A0017001B0017001A002F001B0E
:101500000016001B002F001C002E001B002E001CCC
:10151000002E001C0016001C0014001E002D001CD4
:101520000015001E002D001D001401FC005E001CB3
:101530000015001C002E001D002D001D0015001DB3
:10154000002C001D0015001D0014001D0014001EBD
:10155000002C001D0015001D002C001D002C001E7D
:10156000002C001D002B001F0013001E0013001E86
:10157000002C001D0014001E002C001E001401FD94
:1015800000000000000000000000000000610017E3
:1015900000320019003100190030001B0017001A3A
:1015A000002F001B0017001B0016001C0016001C5B
:1015B000002D001C0016001C002D001C002E001D1C
:1015C000002D001C002D001D0014001D0015001D25
:1015D000002D001D0014001E002C001D001401E44D
:1015E000005D001D002C001D002D001D002C001DA5
:1015F0000015001E002C001E0015001D0014001D0B
:101600000015001E002C001E0014001E002C001DE2
:10161000002B001F002C001E002B001F0014001DBB
:101620000014001E002C001E0013001E002C001EC3
:10163000001301E5000000000000000000000000B1
:101640000062001600320019001900180031001A5B
:10165000001800190017001B002F001A002F001B94
:101660000016001B002F001C0016001B002E001C83
:10167000002E001D002D001C002D001D0015001C5B
:101680000014001E002D001D0014001E002D001D62
:10169000001401E3005E001C002D001D0015001D5C
:1016A000002C001D0015001D0014001D002D001D44
:1016B000002C001D0014001E002C001D0013001F34
:1016C000002C001D002C001F002C001D002B001FF3
:1016D0000014001D0014001E002C001D0014001E2C
:1016E000002C001E001301E40000000000000000B8
:1016F0000000000000620016001A0018001900180F
:1017000000190019001900190018001A0030001AF9
:10171000002F001B0017001A002F001B0016001CD2
:10172000002D001C002E001C002D001C002E001D92
:101730000015001C0015001D002D001C0015001ECA
:10174000002D001D00140214005E001C0015001C7A
:101750000016001C0015001C0016001D0014001DC2
:10176000002D001D002D001D0015001E002C001D69
:101770000014001E002D001D002D001E002C001D59
:10178000002B001F0013001E0013001E002C001D64
:101790000014001E002C001E0013021500000000A3
:1017A000000000000000000000620016001A001790
:1017B000003200180018001A00300019002F001B1A
:1017C0000017001A002F001B0016001B002F001C22
:1017D0000016001B002E001C002E001B002E001CFB
:1017E000002E001D0015001C0014001E002D001D01
:1017F0000014001E002D001D001401E3005E001CFB
:101800000015001D002E001D0014001D002D001DE0
:10181000002D001D0015001D002C001D0014001ED1
:10182000002D001D0013001F002C001D002C001EA9
:10183000002C001D002B001F0014001D0014001EB2
:10184000002C001D0014001E002C001D001401E4DB
:101850000000000000000000000000000062001610
:10186000001A0017003200180018001A0031001981
:101870000017001A0030001A002F001B0016001B72
:10188000002F001C0016001B002F001C002E001C47
:10189000002E001C002D001D0015001C0015001D51
:1018A000002D001D0014001E002D001D001401E37A
:1018B000005E001C0015001C002E001D0014001D01
:1018C000002D001D0014001D002D001D002C001D0A
:1018D0000014001E002D001D0013001F002C001D11
:1018E000002C001E002C001E002C001E0014001DE9
:1018F0000014001E002C001E0013001E002C001DF2
:10190000001401E4000000000000000000000000DE
:101910000062001600320019001900180018001AA1
:10192000003000190017001B002F001A002F001BA9
:101930000016001B002F001C0016001B002E001CB0
:10194000002E001C002E001C002E001D0015001C87
:101950000014001E002D001C0014001E002D001D90
:10196000001401E3005E001C002D001D0015001D89
:101970000014001D002E001D0014001D002D001D70
:10198000002D001D0014001E002C001D0013001F60
:10199000002C001D002C001E002C001D002C001E21
:1019A0000014001D0014001E002C001D0014001E59
:1019B000002C001D001401E40000000000000000E5
:1019C0000000000073656E645F6E756D6265723A4B
:1019D000206E65775F76616C7565200020536F6EB1
:1019E00079204456442F56435220436F6D626F2036
:1019F0004952206465636B20285459504520333187
:101A00002920303531323231200D0A00534F4E59E2
:101A100020333120534C562D443330305020494E22
:101A20004954444546200D0A00534F4E592049520F
:101A3000204D4F444544454620617267756D656E83
:101A400074203D2000536F6E79204952204E554D31
:101A500042200D0A00534F4E59204952204D4F56F7
:101A60004544454620666C61677320617267756DF9
:101A7000656E74203D2000464F525741524420531A
:101A80004F4E59204952204D4F56454445462066F9
:101A90006C61677320617267756D656E74203D209F
:101AA0000073656E64696E6720534F4E592049522A
:101AB00020504C41590D0A00BD8EBD8EBD8EBD8E8D
:101AC000BD8EBD8EBD8EBD8EBD8EBD8EBD8EBD8EBE
:101AD000BD8EBD8EBD8EBD8EBD8EBD8EBD8EBD8EAE
:101AE000BD8EBD8EBD8EBD8EBD8EBD8EBD8EBD8E9E
:101AF000BD8EBD8EBD8EBDD4BD8EBD69BD69BD69B7
:101B0000BD69BD69BD69BD69BD69BD69BD69BD69A5
:101B1000BD69BD69BD69BD69BD69BD69BD69BD6995
:101B2000BD69BD69BD69BD69BD69BD69BD69BD6985
:101B3000BD69BD69BD69BD69BED4BD69424344315B
:101B4000204D4F444544454620666C6167732C2008
:101B5000617267756D656E74200042434431204D9B
:101B60006F766544454620666C6167732C20617210
:101B700067756D656E7420004243443120454449C9
:101B80005444454620666C6167732C20617267750A
:101B90006D656E740D0A002331206770695F63689C
:101BA000616E676564203D2000204243443120423D
:101BB000414E4B31206770695F6368616E67656491
:101BC00020646F5F67706920677069315F6163745B
:101BD00069766520206770695F74656D70200D0AF5
:101BE0000020424344312042414E4B31206770690E
:101BF0005F736F75726365206770695F776F726B73
:101C0000200D0A0010AF028003D38001C39211900F
:101C10000927E0B4010A900927E4F0854399802C54
:101C2000900DADE0FEA3E0FF0FBF00010E7C037D31
:101C3000FFEE5214EF5215900DADECF0A3EDF08CC9
:101C4000168D179009AB12D480E543F0A21192AF24
:101C500022854483854582E49360148544838545C9
:101C600082E493F543121C04784412D4C080E2222B
:101C70009012E7E4F0E54745467003021CFEE54894
:101C80007038AE46AF4774108E148F15FF12D469AA
:101C90008C168D1790A0A412D480FEE493FFEE90D2
:101CA00012E7E09012D612D495EFF0AE46AF47742B
:101CB0000412D4418E468F47803BAE46AF47740A2C
:101CC0008E148F15FF12D4698C168D1790A0A41254
:101CD000D480FEE493FFEE9012E7E09012D612D487
:101CE00095EFF0AE46AF47740A8E148F15FF12D3EE
:101CF000F48C468D479012E7E004F0021C759012B8
:101D0000E7E09012D612D4957430F0E548700B904D
:101D100012E7E00454FE9012E7F09012E7E0C3955A
:101D20004950279012E67401F09012E6E0FE9012FE
:101D3000E7E0F4042549C39E40107430F543121CBB
:101D4000049012E6E02401F050DF9012E7E0601802
:101D50009012E7E014F09012E7E09012D612D495BA
:101D6000E0F543121C0480E2AE4AAF4B8E448F452F
:101D7000121C512285438175430022309857C29826
:101D8000E599B41B08900928E064016002802C905A
:101D90000DCAE0600875994574FF12D3E4C2AF9094
:101DA000D3CC12D39D90D3CC12D39D90D3CC12D34D
:101DB0009D900DAFE0F58175D000229009AAE00456
:101DC000547F9009AAF09009AAE090092912D495AD
:101DD000E599F080A6309949C299900DABE0FEA339
:101DE000E0FF900DADE0FCA3E0FDEF6D7004EE6C44
:101DF00060290FBF00010E7A037BFFEE5212EF52F3
:101E000013900DABEAF0A3EBF08A168B179009AB99
:101E100012D480E0F5438543998006900927740128
:101E2000F022855483855582E0F8A3E0F9A3E0FA17
:101E300085568385578275F000E06830E70375F0BA
:101E400003E0C39840157018A3E0C399400D7010CB
:101E5000A3E0C39A40057008740022740165F02263
:101E6000740265F022855483855582E0F8A3E0F979
:101E7000A3E0FA855683855782E8F0A3E9F0A3EA48
:101E8000F022855483855582E0F8A3E0F9A3E0C3EE
:101E90009401FAE99400F9E8940085548385558209
:101EA000F0A3E9F0A3EAF022855683855782E0A3E8
:101EB000F8E0A3F9E0FA8554838555827C987D96F5
:101EC0007E80121F7BE55B2430F0A37C0F7D427E79
:101ED00040121F7BE55B2430F0A37C017D867EA051
:101EE000121F7BE55B2430F0A37C007D277E10125F
:101EF0001F7BE55B2430F0A37C007D037EE8121F8E
:101F00007BE55B2430F0A37C007D007E64121F7BA8
:101F1000E55B2430F0A37C007D007E0A121F7BE588
:101F20005B2430F0A3EA2430F0A37400F02285543F
:101F300083855582E0F8A3E0F9A3E02401FAE934AF
:101F400000F9E83400855483855582F0A3E9F0A3B5
:101F5000EAF022855483855582E0F8A3E0F9A3E0F6
:101F6000F42401FAE9F43400F9E8F43400855483E8
:101F7000855582F0A3E9F0A3EAF0228859895A8AAC
:101F80005B780079007A007F19C3CA9ECAC99DC9CF
:101F9000C89CC8401ED3C55B33C55BC55A33C55A00
:101FA000C55933C559CA33CAC933C9C833C8DFD9BB
:101FB000021FD7CA2ECAC93DC9C83CC8C3C55B33B6
:101FC000C55BC55A33C55AC55933C559CA33CAC981
:101FD00033C9C833C8DFB2C813C8C913C9CA13CAC2
:101FE00022C0E0C0F0C083C082C0D075D01812D02B
:101FF000C5D0D0D082D083D0F0D0E032FFFFFFFF39
:102000001FFFFF00010032E7563830390503007822
:10201000FFFF53545550FFFFFFFFFFFFFFFFFFFF80
:10202000FFFFFFFFFFFFFFFFFFFFFFFFFFFFFFFFC0
:10203000FFFFFFFFFFFFFFFFFFFFFFFFFFFFFFFFB0
:10204000FFFFFFFFFFFFFFFFFFFFFFFFFFFFFFFFA0
:10205000FFFFFFFFFFFFFFFFFFFFFFFFFFFFFFFF90
:10206000FFFFFFFFFFFFFFFFFFFFFFFFFFFFFFFF80
:10207000FFFFFFFFFFFFFFFFFFFFFFFFFFFFFFFF70
:10208000FFFFFFFFFFFFFFFFFFFFFFFFFFFFFFFF60
:10209000FFFF044E554C4CFFFFFFFFFFFFFFFFFF0C
:1020A000FFFFFFFFFFFFFFFFFFFFFFFFFFFFFFFF40
:1020B000FFFFFFFFFFFFFFFFFFFFFFFFFFFFFFFF30
:1020C000FFFFFFFFFFFFFFFFFFFFFFFFFFFFFFFF20
:1020D000FFFFFFFFFFFFFFFFFFFFFFFFFFFFFFFF10
:1020E000FFFFFFFFFFFFFFFFFFFFFFFFFFFFFFFF00
:1020F000FFFFFFFFFFFFFFFFFFFFFFFFFFFFFFFFF0
:10210000FFFFFFFFFFFFFFFFFFFFFFFFFFFFFFFFDF
:10211000FFFFFF045354444EFFFFFFFFFFFFFFFF8D
:10212000FFFFFFFFFFFFFFFFFFFFFFFFFFFFFFFFBF
:10213000FFFFFFFFFFFFFFFFFFFFFFFFFFFFFFFFAF
:10214000FFFFFFFFFFFFFFFFFFFFFFFFFFFFFFFF9F
:10215000FFFFFFFFFFFFFFFFFFFFFFFFFFFFFFFF8F
:10216000FFFFFFFFFFFFFFFFFFFFFFFFFFFFFFFF7F
:10217000FFFFFFFFFFFFFFFFFFFFFFFFFFFFFFFF6F
:10218000FFFFFFFFFFFFFFFFFFFFFFFFFFFFFFFF5F
:10219000FFFFFFFF0453544C46FFFFFFFFFFFFFF0D
:1021A000FFFFFFFFFFFFFFFFFFFFFFFFFFFFFFFF3F
:1021B000FFFFFFFFFFFFFFFFFFFFFFFFFFFFFFFF2F
:1021C000FFFFFFFFFFFFFFFFFFFFFFFFFFFFFFFF1F
:1021D000FFFFFFFFFFFFFFFFFFFFFFFFFFFFFFFF0F
:1021E000FFFFFFFFFFFFFFFFFFFFFFFFFFFFFFFFFF
:1021F000FFFFFFFFFFFFFFFFFFFFFFFFFFFFFFFFEF
:10220000FFFFFFFFFFFFFFFFFFFFFFFFFFFFFFFFDE
:10221000FFFFFFFFFF0453545254FFFFFFFFFFFF78
:10222000FFFFFFFFFFFFFFFFFFFFFFFFFFFFFFFFBE
:10223000FFFFFFFFFFFFFFFFFFFFFFFFFFFFFFFFAE
:10224000FFFFFFFFFFFFFFFFFFFFFFFFFFFFFFFF9E
:10225000FFFFFFFFFFFFFFFFFFFFFFFFFFFFFFFF8E
:10226000FFFFFFFFFFFFFFFFFFFFFFFFFFFFFFFF7E
:10227000FFFFFFFFFFFFFFFFFFFFFFFFFFFFFFFF6E
:10228000FFFFFFFFFFFFFFFFFFFFFFFFFFFFFFFF5E
:10229000FFFFFFFFFFFF04454E5452FFFFFFFFFF0C
:1022A000FFFFFFFFFFFFFFFFFFFFFFFFFFFFFFFF3E
:1022B000FFFFFFFFFFFFFFFFFFFFFFFFFFFFFFFF2E
:1022C000FFFFFFFFFFFFFFFFFFFFFFFFFFFFFFFF1E
:1022D000FFFFFFFFFFFFFFFFFFFFFFFFFFFFFFFF0E
:1022E000FFFFFFFFFFFFFFFFFFFFFFFFFFFFFFFFFE
:1022F000FFFFFFFFFFFFFFFFFFFFFFFFFFFFFFFFEE
:10230000FFFFFFFFFFFFFFFFFFFFFFFFFFFFFFFFDD
:10231000FFFFFFFFFFFFFF0450524556FFFFFFFF87
:10232000FFFFFFFFFFFFFFFFFFFFFFFFFFFFFFFFBD
:10233000FFFFFFFFFFFFFFFFFFFFFFFFFFFFFFFFAD
:10234000FFFFFFFFFFFFFFFFFFFFFFFFFFFFFFFF9D
:10235000FFFFFFFFFFFFFFFFFFFFFFFFFFFFFFFF8D
:10236000FFFFFFFFFFFFFFFFFFFFFFFFFFFFFFFF7D
:10237000FFFFFFFFFFFFFFFFFFFFFFFFFFFFFFFF6D
:10238000FFFFFFFFFFFFFFFFFFFFFFFFFFFFFFFF5D
:10239000FFFFFFFFFFFFFFFF044E455854FFFFFF05
:1023A000FFFFFFFFFFFFFFFFFFFFFFFFFFFFFFFF3D
:1023B000FFFFFFFFFFFFFFFFFFFFFFFFFFFFFFFF2D
:1023C000FFFFFFFFFFFFFFFFFFFFFFFFFFFFFFFF1D
:1023D000FFFFFFFFFFFFFFFFFFFFFFFFFFFFFFFF0D
:1023E000FFFFFFFFFFFFFFFFFFFFFFFFFFFFFFFFFD
:1023F000FFFFFFFFFFFFFFFFFFFFFFFFFFFFFFFFED
:10240000FFFFFFFFFFFFFFFFFFFFFFFFFFFFFFFFDC
:10241000FFFFFFFFFFFFFFFFFF04504C41593B54FC
:10242000494D4532303B504F57523B54494D453250
:10243000303B504C4159FFFFFFFFFFFFFFFFFFFF05
:10244000FFFFFFFFFFFFFFFFFFFFFFFFFFFFFFFF9C
:10245000FFFFFFFFFFFFFFFFFFFFFFFFFFFFFFFF8C
:10246000FFFFFFFFFFFFFFFFFFFFFFFFFFFFFFFF7C
:10247000FFFFFFFFFFFFFFFFFFFFFFFFFFFFFFFF6C
:10248000FFFFFFFFFFFFFFFFFFFFFFFFFFFFFFFF5C
:10249000FFFFFFFFFFFFFFFFFFFF1C5245544EFFF2
:1024A000FFFFFFFFFFFFFFFFFFFFFFFFFFFFFFFF3C
:1024B000FFFFFFFFFFFFFFFFFFFFFFFFFFFFFFFF2C
:1024C000FFFFFFFFFFFFFFFFFFFFFFFFFFFFFFFF1C
:1024D000FFFFFFFFFFFFFFFFFFFFFFFFFFFFFFFF0C
:1024E000FFFFFFFFFFFFFFFFFFFFFFFFFFFFFFFFFC
:1024F000FFFFFFFFFFFFFFFFFFFFFFFFFFFFFFFFEC
:10250000FFFFFFFFFFFFFFFFFFFFFFFFFFFFFFFFDB
:10251000FFFFFFFFFFFFFFFFFFFFFF044E554D4290
:1025200031FFFFFFFFFFFFFFFFFFFFFFFFFFFFFF89
:10253000FFFFFFFFFFFFFFFFFFFFFFFFFFFFFFFFAB
:10254000FFFFFFFFFFFFFFFFFFFFFFFFFFFFFFFF9B
:10255000FFFFFFFFFFFFFFFFFFFFFFFFFFFFFFFF8B
:10256000FFFFFFFFFFFFFFFFFFFFFFFFFFFFFFFF7B
:10257000FFFFFFFFFFFFFFFFFFFFFFFFFFFFFFFF6B
:10258000FFFFFFFFFFFFFFFFFFFFFFFFFFFFFFFF5B
:10259000FFFFFFFFFFFFFFFFFFFFFFFF054E554D52
:1025A0004232FFFFFFFFFFFFFFFFFFFFFFFFFFFFC5
:1025B000FFFFFFFFFFFFFFFFFFFFFFFFFFFFFFFF2B
:1025C000FFFFFFFFFFFFFFFFFFFFFFFFFFFFFFFF1B
:1025D000FFFFFFFFFFFFFFFFFFFFFFFFFFFFFFFF0B
:1025E000FFFFFFFFFFFFFFFFFFFFFFFFFFFFFFFFFB
:1025F000FFFFFFFFFFFFFFFFFFFFFFFFFFFFFFFFEB
:10260000FFFFFFFFFFFFFFFFFFFFFFFFFFFFFFFFDA
:10261000FFFFFFFFFFFFFFFFFFFFFFFFFF054E551F
:102620004D4233FFFFFFFFFFFFFFFFFFFFFFFFFFF5
:10263000FFFFFFFFFFFFFFFFFFFFFFFFFFFFFFFFAA
:10264000FFFFFFFFFFFFFFFFFFFFFFFFFFFFFFFF9A
:10265000FFFFFFFFFFFFFFFFFFFFFFFFFFFFFFFF8A
:10266000FFFFFFFFFFFFFFFFFFFFFFFFFFFFFFFF7A
:10267000FFFFFFFFFFFFFFFFFFFFFFFFFFFFFFFF6A
:10268000FFFFFFFFFFFFFFFFFFFFFFFFFFFFFFFF5A
:10269000FFFFFFFFFFFFFFFFFFFFFFFFFFFF054EF5
:1026A000554D4234FFFFFFFFFFFFFFFFFFFFFFFF1E
:1026B000FFFFFFFFFFFFFFFFFFFFFFFFFFFFFFFF2A
:1026C000FFFFFFFFFFFFFFFFFFFFFFFFFFFFFFFF1A
:1026D000FFFFFFFFFFFFFFFFFFFFFFFFFFFFFFFF0A
:1026E000FFFFFFFFFFFFFFFFFFFFFFFFFFFFFFFFFA
:1026F000FFFFFFFFFFFFFFFFFFFFFFFFFFFFFFFFEA
:10270000FFFFFFFFFFFFFFFFFFFFFFFFFFFFFFFFD9
:10271000FFFFFFFFFFFFFFFFFFFFFFFFFFFFFF05C3
:102720004E554D4235FFFFFFFFFFFFFFFFFFFFFF4D
:10273000FFFFFFFFFFFFFFFFFFFFFFFFFFFFFFFFA9
:10274000FFFFFFFFFFFFFFFFFFFFFFFFFFFFFFFF99
:10275000FFFFFFFFFFFFFFFFFFFFFFFFFFFFFFFF89
:10276000FFFFFFFFFFFFFFFFFFFFFFFFFFFFFFFF79
:10277000FFFFFFFFFFFFFFFFFFFFFFFFFFFFFFFF69
:10278000FFFFFFFFFFFFFFFFFFFFFFFFFFFFFFFF59
:10279000FFFFFFFFFFFFFFFFFFFFFFFFFFFFFFFF49
:1027A000054E554D4236FFFFFFFFFFFFFFFFFFFFC6
:1027B000FFFFFFFFFFFFFFFFFFFFFFFFFFFFFFFF29
:1027C000FFFFFFFFFFFFFFFFFFFFFFFFFFFFFFFF19
:1027D000FFFFFFFFFFFFFFFFFFFFFFFFFFFFFFFF09
:1027E000FFFFFFFFFFFFFFFFFFFFFFFFFFFFFFFFF9
:1027F000FFFFFFFFFFFFFFFFFFFFFFFFFFFFFFFFE9
:10280000FFFFFFFFFFFFFFFFFFFFFFFFFFFFFFFFD8
:10281000FFFFFFFFFFFFFFFFFFFFFFFFFFFFFFFFC8
:10282000FF054E554D4237FFFFFFFFFFFFFFFFFF44
:10283000FFFFFFFFFFFFFFFFFFFFFFFFFFFFFFFFA8
:10284000FFFFFFFFFFFFFFFFFFFFFFFFFFFFFFFF98
:10285000FFFFFFFFFFFFFFFFFFFFFFFFFFFFFFFF88
:10286000FFFFFFFFFFFFFFFFFFFFFFFFFFFFFFFF78
:10287000FFFFFFFFFFFFFFFFFFFFFFFFFFFFFFFF68
:10288000FFFFFFFFFFFFFFFFFFFFFFFFFFFFFFFF58
:10289000FFFFFFFFFFFFFFFFFFFFFFFFFFFFFFFF48
:1028A000FFFF054E554D4238FFFFFFFFFFFFFFFFC3
:1028B000FFFFFFFFFFFFFFFFFFFFFFFFFFFFFFFF28
:1028C000FFFFFFFFFFFFFFFFFFFFFFFFFFFFFFFF18
:1028D000FFFFFFFFFFFFFFFFFFFFFFFFFFFFFFFF08
:1028E000FFFFFFFFFFFFFFFFFFFFFFFFFFFFFFFFF8
:1028F000FFFFFFFFFFFFFFFFFFFFFFFFFFFFFFFFE8
:10290000FFFFFFFFFFFFFFFFFFFFFFFFFFFFFFFFD7
:10291000FFFFFFFFFFFFFFFFFFFFFFFFFFFFFFFFC7
:10292000FFFFFF05FFFFFFFFFFFFFFFFFFFFFFFFB1
:10293000FFFFFFFFFFFFFFFFFFFFFFFFFFFFFFFFA7
:10294000FFFFFFFFFFFFFFFFFFFFFFFFFFFFFFFF97
:10295000FFFFFFFFFFFFFFFFFFFFFFFFFFFFFFFF87
:10296000FFFFFFFFFFFFFFFFFFFFFFFFFFFFFFFF77
:1040000010AF028003D38001C39208900DDCE0FE64
:10401000A3E0FFAC35AD36EE4204EF4205900DDC77
:10402000ECF0A3EDF0A20892AF2210AF028003D310
:104030008001C39208900DDCE0FEA3E0FFE535F4BB
:10404000FCE536F4FDEE5204EF5205900DDCECF089
:10405000A3EDF0A20892AF22900DDCE0FEA3E0FFFA
:10406000AC35AD36EE5204EF5205ED4C6002D32272
:10407000C322900DDCE0FEA3E0FFAC35AD36EE527E
:1040800004EF5205AA35AB36EDB50306ECB50202D6
:10409000D322C32210AF028003D38001C3920875DC
:1040A0004C0D754DC5754E10754F9112CD96A208E9
:1040B00092AF7E107F9122E539C394025024E539F6
:1040C00020E003C38001D3B39200AE35AF368E4CEF
:1040D0008F4D85374E85384F853A5012CC9CC200A3
:1040E000D32274009010A2F09010A1F09010A0F0D4
:1040F00090109FF090109EF0AE35AF36E53A2FFF4E
:1041000050010E1FBFFF011E8E358F36E53A70033A
:1041100002419C853583853682E09010A3F0783586
:1041200012D4C8153A9010A3E0B43A0280DE901081
:10413000A3E0C39430FE90109EE090109F12D4959F
:10414000EEF0E53A70028054853583853682E09042
:1041500010A3F0783512D4C8153A9010A3E0B43A01
:104160000280DF9010A3E0C3943075F00AA4FFAE84
:10417000F090109EE090109F12D495EFFFE0FCEFBE
:104180002CFE90109EE090109F12D495EEF09010AF
:104190009EE004540390109EF002410C9010A2E0A7
:1041A000D3942350129010A1E0D3943B5009901067
:1041B000A0E0D3943B4002C3229010A2E075F00A25
:1041C00084FF7E00EF90109BF09010A2E075F00A43
:1041D00084ADF07C00ED90109AF09010A1E075F0A5
:1041E0000A84FF7E00EF901099F09010A1E075F026
:1041F0000A84ADF07C00ED901098F09010A0E0756E
:10420000F00A84FF7E00EF901097F09010A0E07508
:10421000F00A84ADF07C00ED901096F090109FE0D5
:1042200075F00A84FF7E00EF901095F090109FE0EB
:1042300075F00A84ADF07C00ED901094F0E539B48F
:10424000021A90109FE0D3941D4002C322754C10B7
:10425000754D9485374E85384F12CF0FD322900D70
:10426000ABE0FEA3E0FF900DADE0FCA3E0FDEF6D41
:104270007004EE6C600280E622853583853682E428
:10428000936016853583853682E493F59974FF1221
:10429000D3E4783512D4C080E080FE2210AF0280D3
:1042A00003D38001C39208900927E0B4010A900962
:1042B00027E4F0853599802C900DADE0FEA3E0FF5A
:1042C0000FBF00010E7C037DFFEE5204EF520590FC
:1042D0000DADECF0A3EDF08C068D079009AB12D478
:1042E00080E535F0A20892AF22853683853782E0DB
:1042F0006013853683853782E0F53512429C783627
:1043000012D4C080E422853683853782E49360141A
:10431000853683853782E493F53512429C783612D0
:10432000D4C080E222E5386015853683853782E087
:10433000F53512429C783612D4C0153880E722E554
:10434000386016853683853782E493F53512429CB2
:10435000783612D4C0153880E6229010B5E4F0E526
:1043600039453870030243E8E53A7038AE38AF3962
:1043700074108E048F05FF12D4698C068D0790A0EF
:10438000A412D480FEE493FFEE9010B5E09010A448
:1043900012D495EFF0AE38AF39740412D4418E3890
:1043A0008F39803BAE38AF39740A8E048F05FF1207
:1043B000D4698C068D0790A0A412D480FEE493FFEC
:1043C000EE9010B5E09010A412D495EFF0AE38AF97
:1043D00039740A8E048F05FF12D3F48C388D39900E
:1043E00010B5E004F002435F9010B5E09010A41205
:1043F000D4957430F0E53A700B9010B5E00454FE9B
:104400009010B5F09010B5E0C3953B50279010B4D4
:104410007401F09010B4E0FE9010B5E0F404253B78
:10442000C39E40107430F53512429C9010B4E024C5
:1044300001F050DF9010B5E060189010B5E014F076
:104440009010B5E09010A412D495E0F53512429C7E
:1044500080E2AE3CAF3D8E368F3712430622853E5A
:104460004C853F4D754E10754FC612CD96900DCFB1
:10447000E07022754C10754D3E853E4E853F4F12C3
:10448000CD53B40110742DF53512429C754C107546
:104490004DC612CE84E540909FF9F82828739010FD
:1044A000C6E0F539753800753A007402F53B753C85
:1044B000A0753DBF12435A9010C7E0F5397538001A
:1044C000753A007402F53B753CA0753DBF12435A26
:1044D0009010C8E0F539753800753A007402F53B64
:1044E000753CA0753DBF12435A8077900DCFE0B464
:1044F0000148754C10754D3E853E4E853F4F12CD9F
:1045000053B40136754C10754DC612CE84754C10DF
:10451000754D38754E10754FC912CD96754C107586
:104520004DC9754E10754FC612CFA9754C10754DFB
:10453000C9754E10754FC612CD96754C10754DB697
:10454000754E10754FC612CDD97536107537B61227
:1045500042E9800E800C800A800880068004800278
:104560008000AE41AF428E368F371243062210AE26
:10457000028003D38001C39208AE36AF37748052F5
:10458000077E00EF4E605B900EDDE014541F900E2E
:10459000DDF0900EDDE07F07900EDF12D404E535EC
:1045A000F0900EDDE07F07900EE012D404E536F0C7
:1045B000A3E537F0900EDDE07F07900EE212D40401
:1045C000E539F0853A4C853B4D900EDDE07F079054
:1045D0000EE312D404AE83AF828E4E8F4F12CD966F
:1045E0008059900EDEE07F07900EDF12D404E5358F
:1045F000F0900EDEE07F07900EE012D404E536F076
:10460000A3E537F0900EDEE07F07900EE212D404AF
:10461000E539F0853A4C853B4D900EDEE07F079002
:104620000EE312D404AE83AF828E4E8F4F12CD961E
:10463000900EDEE004541F900EDEF0A20892AE222F
:1046400074009010CCF09010CDE535F0A3E536F075
:10465000744D9010CFF8E4F0E8A3F09010CFE0FE96
:10466000A3E0FF8E4C8F4D754E10754FCC12CEAC23
:10467000754C10754DCC12CE5F10AF028003D38005
:1046800001C39208754C0D754DB6E5377F03900D4B
:10469000B912D404AE83AF828E4E8F4F12CD96E501
:1046A000377F03900DB912D404AE83AF828E4C8F46
:1046B0004D754E10754FCC12CC6CE537900DBF1276
:1046C000D4957400F0A20892AF228538358539362A
:1046D000753700124640900DBFE0700280F82275D9
:1046E0003502753610124072C0D0900EDDE0FE909B
:1046F0000EDEE0B50603C38001D392F0D0D072F095
:10470000500B7539647538001246CA80D29010D1AA
:10471000E4F0A304F09010D1E0FEA3E0FF900DECD4
:10472000E0BE003E9F403B7539C87538001246CA4E
:10473000753610753500124058C0D0753502753683
:1047400000124058B392F0D0D0B382F05002D3227E
:104750009010D2E02401F050079010D1E03400F026
:1047600050B37412900DCCF0124094C006C007D024
:1047700007D0068E4C8F4D754E10754F7B12CD961F
:10478000C3229010D3E4F0A304F09010D3E0FEA372
:10479000E0FF900DEBE0BE002B9F402875350275C1
:1047A00036001240585002D3227539647538001211
:1047B00046CA9010D4E02401F050079010D3E034A2
:1047C00000F050C674FC900DCCF0124094C006C0AE
:1047D00007D007D0068E4C8F4D754E10754F7B124B
:1047E000CD96C3227403900010F0900003E4F09083
:1047F0000DCEE4F07430900001F8E4F0E8A3F090FE
:1048000000047401F07432900005F8E4F0E8A3F0BD
:1048100090000A7430F0A37439F090000C7401F029
:10482000740290000DF074C890000EF8E4F0E8A354
:10483000F07403900011F02274199010D7F09010CA
:10484000D57401F09010D5E0D39404504FD2A790C6
:1048500010D67401F09010D6E0FE9010D7E0C39E01
:10486000400E74FA12D3E49010D6E02401F050E523
:10487000C2A79010D67401F09010D6E0FE9010D729
:10488000E0C39E400E74FA12D3E49010D6E02401E7
:10489000F050E59010D5E02401F050A8C2A722E521
:1048A00035642C6023E5356420601DE535640860BF
:1048B00017E535647F6011E5356409600BE5356403
:1048C0000D6005E535B40A02D322C322740E90129E
:1048D00011F0901212E4F0901213E4F0A3F0901291
:1048E00011E0F54C901212E0F54D901213E0F54EE8
:1048F000A3E0F54F901215E0F55012CC4E90121631
:10490000F07536A07537D5124306901216E0F539CA
:10491000753800753A007402F53B753CA0753DB4DE
:1049200012435A901213E4F0A304F0901211E0F530
:104930004C901212E0F54D901213E0F54EA3E0F505
:104940004F901215E0F55012CC4E901216F07536BD
:10495000A07537E4124306901216E0F53975380059
:10496000753A007402F53B753CA0753DB412435A8C
:104970007402901213F8E4F0E8A3F0901211E0F53D
:104980004C901212E0F54D901213E0F54EA3E0F5B5
:104990004F901215E0F55012CC4E901216F075366D
:1049A000A07537F6124306901216E0F539753800F7
:1049B000753A007402F53B753CA0753DB412435A3C
:1049C00022222222223003139011FFE090A017F838
:1049D00028287380048002800080002222C2AFE574
:1049E0008114901217F0901217E0F8760008760004
:1049F000223003119011FEE0F8A3E0901089C8F076
:104A0000A3C8F0801F901089E0FEA3E0FF8E388FCE
:104A100039901210E0F53A7404F53B753CA0753DF1
:104A2000B412435A223003129011FFE0900DCAF0E5
:104A3000900DCAE0900004F08038900DCAE0F5397E
:104A4000753800901210E0F53A7401F53B753CA002
:104A5000753DB712435A900004E0F539753800905F
:104A60001210E0F53A7401F53B753CA0753DB412A7
:104A7000435A229011FEE0F8A3E0901218C8F0A368
:104A8000C8F090121BE4F090121BE0D39403506A1C
:104A9000901218E0FEA3E0FF8E388F39753A00744B
:104AA00004F53B753CA0753DBB12435A90121AE4C5
:104AB000F090121AE0D3940F502B90121812D45D7C
:104AC000E0F539753800753A007402F53B753CA085
:104AD000753DB712435A90121812002690121AE030
:104AE0002401F050CC7536A07537B412430612423B
:104AF0005E90121BE02401F0508D2230030A9011C9
:104B0000FFE09011F3F0801C9011F3E0F539753857
:104B100000901210E0F53A7401F53B753CA0753D2C
:104B2000B412435A229011F3E4F0229011F374016D
:104B3000F022900DD0E070267535047E017F008E46
:104B4000368F377480F539753800753A10753B32F9
:104B500012456E7539C87538001246CA805C12401D
:104B600094C006C007754C11754DFDD007D0068E58
:104B70004E8F4F12CD53C0E0D006EE90A023F82800
:104B8000287380367535047402F537753600741550
:104B9000F539753800753A11753BFD12456E801A6E
:104BA0007535047403F5377536007415F5397538A5
:104BB00000753A11753BFD12456E22300311A209B2
:104BC000B34006A209B3B35004A2099202801CE4C8
:104BD000A20233F539753800901210E0F53A7401ED
:104BE000F53B753CA0753DB412435A2230030A9040
:104BF00011FFE0900DCCF08045900DCCE0F53975BB
:104C00003800901210E0F53A7405F53B753CA0753C
:104C10003DB712435A753E10753F7B901210E0F578
:104C2000407541A07542B412445E900DCCE4F0751D
:104C30004C10754D3E754E10754F7B12CD9622303F
:104C4000030A9011FFE0900DCCF08039900DCCE07C
:104C5000F539753800901210E0F53A7405F53B759A
:104C60003CA0753DB412435A74009011EFF0900DC2
:104C7000CDF0900DCCF0754C10754D3E754E107505
:104C80004F7B12CD9622C2AFE5811490121CF0909A
:104C9000121CE0F8760008760022900DD0E0B401F6
:104CA0001D7535047400F5377536007415F53975C2
:104CB0003800753A10753B3212456E024D44753519
:104CC000047E017F008E368F377480F53975380089
:104CD000753A10753B3212456E753964753800129D
:104CE00046CA300345124094C006C007754C117582
:104CF0004DFDD007D0068E4E8F4F12CD53C0E0D061
:104D000006EE6402601C7535047402F537753600D2
:104D10007415F539753800753A11753BFD12456EFD
:104D200080067404900DCCF0801A7535047400F57B
:104D3000377536007415F539753800753A10753BBE
:104D40003212456E227535037400F53775360074DE
:104D50008CF539753800753A10753B3212456E2264
:104D60003003219011FFE0641960079011FFE0B457
:104D70001E0A9011FFE0900DD3F080067404900D90
:104D8000CCF0801C900DD3E0F539753800901210EE
:104D9000E0F53A7401F53B753CA0753DB412435AF9
:104DA0002230033E754C11754DFD754E10754F5FE9
:104DB00012CD96754C11754DFD754E0D754FC51282
:104DC000CD96754C11754DFD754E10754F5C12CD1D
:104DD00096754C11754DFD754E0D754FC112CD96E2
:104DE000801E124094C006C007D007D0068E3E8FAA
:104DF0003F901210E0F5407541A07542B412445E38
:104E0000223003119011FEE0F8A3E0900005C8F0F5
:104E1000A3C8F0801F900005E0FEA3E0FF8E388F4E
:104E200039901210E0F53A7402F53B753CA0753DDF
:104E3000B412435A2230030A9011FFE0900EDAF0C8
:104E4000801C900EDAE0F539753800901210E0F50C
:104E50003A7401F53B753CA0753DB412435A2230BB
:104E6000030E9011FFE090106DF0900ED6F0801CB4
:104E7000900ED6E0F539753800901210E0F53A74CE
:104E800001F53B753CA0753DB412435A227536A11D
:104E9000753708124306900E20E0F5397538007515
:104EA0003A017401F53B753CA0753DB712435A9029
:104EB0000E24E0F539753800753A007401F53B753C
:104EC0003CA0753DB712435A900E25E0F539753870
:104ED00000753A007401F53B753CA0753DB712436F
:104EE0005A900E27E0F539753800753A007401F5CF
:104EF0003B753CA0753DB412435A2290121DE4F05C
:104F000090121DE0D394FF501A90121DE090106D86
:104F1000F07539647538001246CA90121DE02401FC
:104F2000F050DD740090106DF0900ED6F0222274D7
:104F3000009011EFF0900DCDF0900DCCF07400903A
:104F40000DD6F0900DD9F0900DDAF0900DD7F090CD
:104F50000DCFE070757535017400F537753600902A
:104F60000DCEE0F539753800753A10753B321245B3
:104F70006E7536A175373A1243067538077539D004
:104F80001246CA900DCEE0F539753800753A0174B5
:104F900002F53B900DD1E0FEA3E0FF8E3C8F3D1269
:104FA000435A7536A175374D1243067535027400A4
:104FB000F537753600900DCEE0F539753800753A45
:104FC00010753B3212456E025065900DCCE0B41E58
:104FD000237535037400F5377536007401F539759E
:104FE0003800753A10753B3212456E7538017539C7
:104FF000F41246CA900DCCE4F0900DCDE4F0753576
:10500000047400F537753600740AF5397538007583
:105010003A10753B3212456E1247824006124782A3
:1050200040012275381275391E1246CA753812753C
:10503000391E1246CA7535047E017F008E368F37C1
:105040007480F539753800753A10753B3212456E2B
:10505000900DD7E0700674FD900DCCF0900EDBE063
:10506000B4010280F7227535037400F537753600F8
:105070007480F539753800753A10753B3212456EFB
:10508000227535037400F5377536007450F539759F
:105090003800753A10753B3212456E229009AAE02D
:1050A00004547F901221F8E4F0E8A3F0901221E07C
:1050B000FEA3E0FF9009A9E06F4E603F900929121E
:1050C000D480E0901223F0901223E0F53512429C38
:1050D000901223E0B40D07740AF53512429C901229
:1050E00021E0FEA3E0FF0FBF00010E747F52077E98
:1050F00000901221EEF0A3EFF080B17536A0753765
:10510000B4124306222222223003519011FFE09074
:105110001227F0901227E0B40121D2A79012277431
:1051200001F0901227E0D39464500E74FA12D3E485
:10513000901227E02401F050E9801FC2A7901227A7
:105140007401F0901227E0D39464500E74FA12D3D5
:10515000E4901227E02401F050E98003124838223D
:10516000754C12754D0D754E10754F3E12CD53B4E2
:105170000111754C12754D0D12CDB390120CE090CB
:105180000EC9F02230033F754C11754DFD754E125E
:10519000754F0D12CD96754C12754D0D12CDB39005
:1051A0000DCAE06012753E12753F0D7540017541E4
:1051B000A07542B412445E900EC9E090120BF8E460
:1051C000F0E8A3F08015753E12753F0D901210E0C7
:1051D000F5407541A07542B412445E227536A17542
:1051E0003750124306753501753600124058E433C6
:1051F000F539753800901210E0F53A7401F53B75F9
:105200003CA0753DB712435A753502753600124001
:1052100058E433F539753800901210E0F53A74010E
:10522000F53B753CA0753DB712435A753510753680
:1052300000124058E433F539753800901210E0F54B
:105240003A7401F53B753CA0753DB712435A900D79
:10525000CFE0F539753800901210E0F53A7401F599
:105260003B753CA0753DB712435A7536A175378919
:1052700012430690000DE0F539753800753A017457
:1052800002F53B753CA0753DB712435A900E1FE0E6
:10529000F539753800753A017402F53B753CA07517
:1052A0003DB712435A900E3FE0F539753800753A14
:1052B000017401F53B753CA0753DB412435A22754B
:1052C0004C11754DF7754E11754FFD12CC6C227552
:1052D0004C11754DFA754E11754FFD12CC6C229024
:1052E0000DCAE070030253777441F53512429C7485
:1052F0005FF53512429C901228E4F0901228E0D31A
:10530000941E5019901228E0900FE512D495E0F504
:105310003512429C901228E02401F050DE740DF505
:105320003512429C740AF53512429C7453F53512BD
:10533000429C745FF53512429C901228E4F0901262
:1053400028E0D3941E5019901228E090100512D432
:1053500095E0F53512429C901228E02401F050DED1
:10536000740DF53512429C740AF53512429C75365F
:10537000A17537B3124306900ECCE0F53512429C6E
:10538000742CF53512429C900ECDE0F53512429CFE
:10539000742CF53512429C900ECEE0F53512429CED
:1053A000742CF53512429C900ECFE0F53512429CDC
:1053B000742CF53512429C900ED0E0F53512429CCB
:1053C000742CF53512429C900ED1E0F53512429CBA
:1053D000742CF53512429C900ED2E0F53512429CA9
:1053E000740DF53512429C740AF53512429C2275F3
:1053F0003502753600124058500B7536A17537D4FA
:1054000012430680097536A17537DD124306223036
:10541000031C7535037400F5377536009011FFE0F5
:10542000F539753800753A10753B3212456E2230E9
:10543000031C7535047400F5377536009011FFE0D4
:10544000F539753800753A10753B3212456E229069
:105450000DCAE060097536A17537E6124306753549
:10546000037400F537753600748DF539753800759D
:105470003A10753B3212456E2230031A75350374AB
:1054800000F5377536007453F539753800753A10E4
:10549000753B3212456E2230031A7535037400F5E0
:1054A000377536007445F539753800753A10753B17
:1054B0003212456E22900DCAE060227536A1753712
:1054C000F7124306900E3FE0F539753800753A0142
:1054D0007401F53B753CA0753DB412435A30033757
:1054E0009011FFE0901229F0901229E07011754C94
:1054F00010754D3E754E0E754F3812CD9680169034
:105500001229E0B4010F754C10754D44754E0E759F
:105510004F3812CD96800F754C10754D32754E0E6A
:10552000754F3812CD967535037400F53775360012
:10553000744AF539753800753A0E753B3812456E68
:10554000227535037400F5377536007452F53975D8
:105550003800753A10753B3212456E22900DCAE044
:1055600060097536A275371D124306753503740040
:10557000F537753600744DF539753800753A107584
:105580003B3212456E22900DCAE060097536A27555
:10559000372E1243067535037400F53775360074DF
:1055A0004EF539753800753A10753B3212456E224A
:1055B000900DCAE060097536A275373F1243067533
:1055C00035037400F5377536007416F539753800F3
:1055D000753A10753B3212456E227535037400F52D
:1055E000377536007417F539753800753A10753B04
:1055F0003212456E22900DCAE060097536A27537E9
:10560000501243067535037400F537753600744F34
:10561000F539753800753A10753B3212456E2275B2
:1056200035037400F5377536007424F53975380084
:10563000753A10753B3212456E227535037400F5CC
:10564000377536007425F539753800753A10753B95
:105650003212456E227535037400F53775360074C5
:1056600049F539753800753A10753B3212456E228E
:10567000900DCEE0B4081C7535047400F53775360E
:1056800000740AF539753800753A10753B321245C9
:105690006E801A7535037400F537753600741CF585
:1056A00039753800753A10753B3212456E227535E2
:1056B000037400F5377536007418F53975380075C0
:1056C0003A10753B3212456E227535037400F5377A
:1056D0007536007419F539753800753A10753B3216
:1056E00012456E227535037400F537753600741A4D
:1056F000F539753800753A10753B3212456E2275D2
:1057000035037400F537753600741BF539753800AC
:10571000753A10753B3212456E227535037400F5EB
:1057200037753600748EF539753800753A10753B4B
:105730003212456E227535037400F53775360074E4
:105740003DF539753800753A10753B3212456E22B9
:105750007535037400F5377536007434F5397538CE
:1057600000753A10753B3212456E22900DCAE0600A
:10577000097536A275376112430630030A9011FE8F
:10578000E0F53CA3E0F53D7535097400F537753655
:1057900000AE3CAF3D8E388F39753A10753B3212F2
:1057A000456E22300371754C11754DFD754E0E75A9
:1057B0004F3812CD967535037402F537753600747F
:1057C00046F539753800753A10753B3212456E75DD
:1057D00039C87538001246CA7535037402F5377535
:1057E00036007437F539753800753A0E753B381246
:1057F000456E7538077539D01246CA753503740081
:10580000F5377536007413F539753800753A10752B
:105810003B3212456E801A7535037400F5377536C4
:10582000007446F539753800753A10753B321245EB
:105830006E22754C10754D3E754E0E754F3812CD5B
:1058400096754C11754DFD754E0E754F3812CD96EF
:105850007535037400F5377536007437F5397538CA
:1058600000753A0E753B3812456E22754C11754D18
:10587000FD754E0E754F3812CD967535037400F5D3
:1058800037753600747FF539753800753A0E753BFB
:105890003812456E22300306A2099202802BE4A240
:1058A0000233F539753800901210E0F53A7401F5BD
:1058B0003B753CA0753DB412435A900DCAE0600997
:1058C0007536A275377712430622900DCAE0601331
:1058D00075994E743212D3E475990D743212D3E473
:1058E00075990A743212D3E42222900DD0E0B401EB
:1058F0001D7535047400F5377536007480F53975FB
:105900003800753A10753B3212456E02599D3003CE
:105910004B124094C006C007754C11754DFDD00761
:10592000D0068E4E8F4F12CD53C0E0D006EE6402EB
:105930006022900DC47401F07535047402F537755A
:1059400036007480F539753800753A11753BFD12D3
:10595000456E80067404900DCCF08041753502755B
:105960003600124058501C7535047400F5377536F2
:10597000007480F539753800753A10753B32124560
:105980006E801A7535047400F53775360074FFF5AE
:1059900039753800753A10753B3212456E229011F8
:1059A000FFE0C39480C4540F90A02CF82828738083
:1059B0005A9011FFE0540790A044F8282873C29031
:1059C000801AC2918016C2928012C293800EC29435
:1059D000800AC2958006C2968002C297802D802BD5
:1059E0009011FFE0540790A05CF8282873C2B080A3
:1059F0001AC2B18016C2B28012C2B3800EC2B48085
:105A00000AC2B58006C2B68002C2B7229011FE1249
:105A1000D45DE0F539753800901210E0F53A740164
:105A2000F53B753CA0753DB412435A22E580F5392B
:105A3000753800753A007402F53B753CA2753D9DC2
:105A400012435AE590F539753800753A007402F53D
:105A50003B753CA2753DA712435AE5A0F539753850
:105A600000753A007402F53B753CA2753DB11243D6
:105A70005AE5B0F539753800753A007402F53B7592
:105A80003CA2753DBB12435A7536A27537C6124308
:105A900006E4A29133F539753800753A007402F5C1
:105AA0003B753CA0753DB712435AE4A29233F539D9
:105AB000753800753A007402F53B753CA0753DB72A
:105AC00012435AE4A29333F539753800753A0074DD
:105AD00002F53B753CA0753DB712435AE4A29433DE
:105AE000F539753800753A007402F53B753CA075C0
:105AF0003DB712435AE4A29533F539753800753A2B
:105B0000007402F53B753CA0753DB712435AE4A200
:105B1000A033F539753800753A007402F53B753CD1
:105B2000A0753DB712435AE4A2A133F53975380088
:105B3000753A007402F53B753CA0753DB712435AA7
:105B4000E4A2A233F539753800753A007402F53BCA
:105B5000753CA0753DB712435A7536A07537B7121C
:105B600043067536A07537B7124306E4A2A333F592
:105B700039753800753A007402F53B753CA0753DE7
:105B8000B712435AE4A2A433F539753800753A00C8
:105B90007402F53B753CA0753DB712435AE4A2A5CB
:105BA00033F539753800753A007402F53B753CA041
:105BB000753DB712435AE4A2A633F539753800751E
:105BC0003A007402F53B753CA0753DB712435AE4A8
:105BD000A2B333F539753800753A007402F53B7598
:105BE0003CA0753DB712435AE4A2B533F539753878
:105BF00000753A007402F53B753CA0753DB7124341
:105C00005AE4A2B633F539753800753A007402F5D6
:105C10003B753CA0753DB712435AE4A2B733F53942
:105C2000753800753A007402F53B753CA0753DB7B8
:105C300012435A7536A07537B41243062230034515
:105C4000124094C006C007754C11754DFDD007D0A9
:105C5000068E4E8F4F12CD53C0E0D006EE64026028
:105C60001C7535047402F537753600740AF53975FC
:105C70003800753A11753BFD12456E80067404902C
:105C80000DCCF0801A7535047400F5377536007444
:105C90000AF539753800753A10753B3212456E2297
:105CA0009011FE12D45DA883A9829011FDE0888333
:105CB0008982F0223003119011FEE0F8A3E0900DEC
:105CC000B4C8F0A3C8F0801C900DB4E0FEA3E0FFC0
:105CD0008E388F39753A017406F53B753CA0753DD9
:105CE000B412435A2290106BE4F0227536A2753735
:105CF000FB1243067536A3753711124306E580F58E
:105D000039753800753A007402F53B753CA0753D55
:105D1000B712435AE590F539753800753A007402A8
:105D2000F53B753CA0753DB712435AE5A0F53975B2
:105D30003800753A007402F53B753CA0753DB7120A
:105D4000435AE5B0F539753800753A007402F53BF1
:105D5000753CA0753DB712435AE5A8F53975380072
:105D6000753A007402F53B753CA0753DB712435A75
:105D70007420F53512429CE598F539753800753A6E
:105D8000007402F53B753CA0753DB712435A753659
:105D9000A3753751124306E588F539753800753A11
:105DA000007402F53B753CA0753DB712435A753639
:105DB000A3753754124306E5C8F539753800753AAE
:105DC000007402F53B753CA0753DB712435A753619
:105DD000A3753758124306E589F539753800753AC9
:105DE000007402F53B753CA0753DB712435A7536F9
:105DF000A375375C124306E5C9F539753800753A65
:105E0000007402F53B753CA0753DB712435A7536D8
:105E1000A3753760124306E4A2AD33F53975380037
:105E2000753A007401F53B753CA0753DB712435AB5
:105E30007536A3753763124306E4A2E833F5397566
:105E40003800753A007401F53B753CA0753DB712FA
:105E5000435A7536A3753766124306E5B8F53975AA
:105E60003800753A007402F53B753CA0753DB712D9
:105E7000435A7536A3753767124306E5B7F539758A
:105E80003800753A007402F53B753CA0753DBF12B1
:105E9000435A7536A3753769124306E4A2AE33F54B
:105EA00039753800753A007401F53B753CA0753DB5
:105EB000B712435A7536A07537B41243067536A328
:105EC00075376B124306E5C1F539753800753A0030
:105ED0007402F53B753CA0753DB712435A7536A365
:105EE000753779124306E5C0F539753800753A0003
:105EF0007402F53B753CA0753DB712435A7536A048
:105F00007537B4124306125CE52230030A9011FF84
:105F1000E090000CF0803B7536A375377C12430689
:105F200090000CE0F539753800753A017402F53BC4
:105F3000753CA0753DB712435A901087E0F539754E
:105F40003800753A017402F53B753CA0753DB412FA
:105F5000435A227535037400F5377536007401F520
:105F600039753800753A10753B3212456E7536A09A
:105F70007537B4124306229011FFE0F88639753860
:105F800000901210E0F53A7401F53B753CA0753DA8
:105F9000B412435A2230030A900E4CE09011F6F0EE
:105FA00080129011F6E0F53512429C7536A07537D7
:105FB000B412430622300311754C11754DFD754E18
:105FC0000D754FF712CD968015753E0D753FF79004
:105FD0001210E0F5407541A07542B412445E229063
:105FE0000DCAE0B4010280030260759011FEE0F872
:105FF000A3E090122CC8F0A3C8F090122FE4F09008
:10600000122FE0D39403506B90122CE0FEA3E0FF1C
:106010008E388F39753A007404F53B753CA0753D98
:10602000BB12435A90122EE4F090122EE0D3940F3C
:10603000502C90122C12D45DE493F539753800750C
:106040003A007402F53B753CA0753DB712435A9077
:10605000122C12002690122EE02401F050CB75363F
:10606000A07537B412430612425E90122FE024014D
:10607000F0508C80209011FE12D45DE493F53975B8
:106080003800901210E0F53A7401F53B753CA075AC
:106090003DB712435A229011FFE0C39480C4540FBD
:1060A00090A038F8282873805A9011FFE054079088
:1060B000A074F8282873D290801AD2918016D292B8
:1060C0008012D293800ED294800AD2958006D29606
:1060D0008002D297802D802B9011FFE0540790A072
:1060E0008CF8282873D2B0801AD2B18016D2B28030
:1060F00012D2B3800ED2B4800AD2B58006D2B68056
:1061000002D2B7223003119011FEE0F8A3E0900F05
:10611000BFC8F0A3C8F0801F900FBFE0FEA3E0FF50
:106120008E388F39901210E0F53A7401F53B753CCA
:10613000A0753DB412435A223003119011FEE0F8CD
:10614000A3E090000EC8F0A3C8F0801C90000EE001
:10615000FEA3E0FF8E388F39753A017405F53B7563
:106160003CA0753DB412435A22900DCAE0600975F7
:1061700036A3753792124306300345124094C00689
:10618000C007754C11754DFDD007D0068E4E8F4F50
:1061900012CD53C0E0D006EE6402601C7535067463
:1061A00002F5377536007410F539753800753A11F7
:1061B000753BFD12456E80067404900DCCF080296D
:1061C000900DCAE060097536A375379F12430675B6
:1061D00035067400F5377536007410F539753800DA
:1061E000753A10753B3212456E22A203B340117509
:1061F0004C11754DFD754E11754FF712CD968015EA
:10620000753E11753FF7901210E0F5407541A0758D
:1062100042B412445E22A203B34011754C11754D75
:10622000FD754E11754FFA12CD968015753E11759C
:106230003FFA901210E0F5407541A07542B4124447
:106240005E227535037400F537753600740CF53928
:10625000753800753A10753B3212456E22300312C4
:106260009011FFE090000DF09011FFE0901073F09E
:106270008038901073E0F539753800901210E0F511
:106280003A7402F53B753CA0753DB712435A900035
:106290000DE0F539753800901210E0F53A7402F50A
:1062A0003B753CA0753DB412435A22900DD0E0B42A
:1062B000011D7535047401F5377536007415F5390F
:1062C000753800753A10753B3212456E026355758C
:1062D00035047E017F008E368F377480F53975382E
:1062E00000753A10753B3212456E7539C875380025
:1062F0001246CA300345124094C006C007754C11BF
:10630000754DFDD007D0068E4E8F4F12CD53C0E095
:10631000D006EE6401601C7535047403F5377536DC
:10632000007415F539753800753A11753BFD124545
:106330006E80067404900DCCF0801A7535047401DB
:10634000F5377536007415F539753800753A1075DE
:106350003B3212456E227535047400F537753600F0
:1063600074FFF539753800753A10753B3212456E79
:1063700022753E0E753F0D901210E0F5407541A05C
:106380007542B412445E2230030A9011FFE090007F
:1063900011F08019900011E0F539753800753A0157
:1063A0007403F53B753CA0753DB412435A22754CFD
:1063B00010754D3E754E0E754F3812CD9690108D5E
:1063C000E0900E3AF0753E0E753F3875400175410C
:1063D000A07542B412445E7535037400F537753606
:1063E000007437F539753800753A0E753B3812452B
:1063F0006E90108DE004F090108DE0FE900011E0A2
:10640000C39E500690108D7401F02212425EC2AFFE
:106410007400F54C754D01754E20754F007400F5F4
:106420005012CC4E900DB0F0D2AF2212425EC2AFED
:10643000740EF54C754D0285354E85364FE537F5B2
:106440005012CC4E901230F0D2AF901230E0229029
:106450000DCAE0900004F0900DCEE0900000F090A6
:106460000E41E0900007F0900E42E0900008F0909E
:106470000E43E0900009F07536A37537B11243065C
:1064800012640B7536A37537C01243067536A375B3
:1064900037D2124306901231E4F0A3F0901231E0AB
:1064A000FEA3E0FF7426C39F74099E500302654A51
:1064B0007C007D00ED2FFFEC3EFE7866A60608A668
:1064C00007901231E0FCA3E0FD8C068D07902000C0
:1064D00012D480AA83AB828A358B3678668683088D
:1064E0008682E0F53712642B60277536A37537E195
:1064F000124306901231E0FEA3E0FF8E388F39750B
:106500003A007404F53B753CA0753DB412435A80C3
:1065100039900DCAE0B4031D78668683088682E050
:10652000F539753800753A007401F53B753CA07576
:106530003DB712435A901232E02401F050079012F6
:1065400031E03400F0400302649C7536A37537F5E2
:1065500012430622755C20755D00755E00755F0054
:1065600075600975612712D31222300364901235C9
:106570007401F0901235E0D394055053901235E039
:1065800090A0C612D424E493FC740193FD9011FEF4
:10659000E0FEA3E0FFEDB50724ECB50620C28E9027
:1065A0001235E090A0C093F58BF58DD28E90123508
:1065B000E0900010F090106EF012644F227536A437
:1065C000753706124306901235E02401F050A4807E
:1065D0003990106EE090A0C612D424783812D49E60
:1065E000753A017401F53B753CA0753DB712435AED
:1065F000900DCAE0600B7536A475371A12430680F9
:10660000097536A07537B412430622753504740037
:10661000F5377536007416F539753800753A10750A
:106620003B3212456E22753E10753F5C901210E0B1
:10663000F5407541A475424812445E753E0D753FA4
:10664000C1901210E0F5407541A475425712445EA6
:10665000753E10753F62901210E0F5407541A475CB
:10666000426612445E753E10753F38901210E0F598
:10667000407541A475427612445E753E10753F5FC9
:10668000901210E0F5407541A475428512445E7584
:106690003E10753F65901210E0F5407541A47542BB
:1066A0009412445E901236E4F0901236E0D39414C3
:1066B0005030901236E0F4042414900FE512D49573
:1066C000E0C39430F539753800753A007402F53B33
:1066D000753CA0753DB712435A901236E02401F084
:1066E00050C77536A47537A41243062222900DCAEE
:1066F000E060097536A47537B61243067535047423
:1067000000F5377536007433F539753800753A1170
:10671000753BFD12456E22900DCAE060097536A4E6
:106720007537C71243067535037400F537753600A3
:10673000744CF539753800753A10753B3212456E58
:1067400022900DCAE060097536A47537DC12430645
:106750007535037400F537753600744BF5397538A7
:1067600000753A10753B3212456E22900DCAE060FA
:10677000097536A47537F11243067535037400F5B3
:10678000377536007451F539753800753A10753B18
:106790003212456E2230031A7535117536FD753784
:1067A0000B7538117539FD740BF53A7400F53B1211
:1067B00066EC227536A57537061243067536A57543
:1067C0003718124306900E40E0F539753800753AD7
:1067D000017401F53B753CA0753DB412435A753602
:1067E000A5753725124306900DB4E0FEA3E0FF8E99
:1067F000388F39753A017406F53B753CA0753DB488
:1068000012435A7536A5753731124306901082E04F
:10681000F539753800753A017401F53B753CA07582
:106820003DB412435A22124094C006C007D007D08C
:10683000068E3E8F3F901210E0F5407541A07542E4
:10684000B912445E7535027536001240585009740D
:1068500031F53512429C80077430F53512429C7434
:106860002CF53512429C900E12E0F53975380090E7
:106870001210E0F53A7402F53B753CA0753DB91273
:10688000435A900DCCE0F539753800753A0174051E
:10689000F53B753CA0753DBF12435A7536A575375B
:1068A0003E124306900DCCE4F0900DCDE4F0901133
:1068B000EFE4F022300A1C7535047411F537753693
:1068C000007401F539753800753A10753B32124580
:1068D0006E801A7535047410F5377536007401F53D
:1068E00039753800753A10753B3212456E22A20A8E
:1068F000B340247535047421F5377536009011FFC7
:10690000E075F002A4FFAEF08E388F39753A10753D
:106910003B3212456E80227535047420F53775368A
:10692000009011FFE075F002A4FFAEF08E388F39B1
:10693000753A10753B3212456E22754C11754DFD3E
:10694000754E12754F3A12CD96900DD0E0B4013DC0
:10695000900DCAE0601B7536A57537411243067568
:106960003E12753F3A7540017541A07542B412441C
:106970005E7535047402F5377536007448F539755F
:106980003800753A12753B3A12456E80002230038A
:106990000A9011FFE0900DECF0801C900DECE0F5FA
:1069A00039753800901210E0F53A7403F53B753CE8
:1069B000A0753DB412435A22300346124094C006DB
:1069C000C007754C11754DFDD007D0068E4E8F4F08
:1069D00012CD53C0E0D006EE6402601D7535047E12
:1069E000017F028E368F377480F539753800753A1D
:1069F00011753BFD12456E80067404900DCCF0803D
:106A0000267E017F008E358F3612402A7535047E32
:106A1000017F008E368F377480F539753800753AEE
:106A200010753B3212456E22E4A28033F539753879
:106A300000901210E0F53A7401F53B753CA0753DED
:106A4000B412435A22200303026B5B755CA5755D8B
:106A500055901205E0FEA3E0FF900E4812D480ACE2
:106A600083AD828C5E8D5F75610475600012D265A6
:106A7000EFB4FF0DEEB4FF097536A5753759124313
:106A800006755CA5755D6E901205E0FEA3E0FF90B3
:106A90000E4812D480AC83AD828C5E8D5F7561042C
:106AA00075600012D265EFB4FF0DEEB4FF097536C4
:106AB000A5753772124306755CA5755D8790120542
:106AC000E0FEA3E0FF900E4812D480AC83AD828C30
:106AD0005E8D5F75610475600012D265EFB4FF0DC5
:106AE000EEB4FF097536A575378B124306755CA5A4
:106AF000755DA0901205E0FEA3E0FF900E4812D451
:106B000080AC83AD828C5E8D5F7561047560001210
:106B1000D265EFB4FF0DEEB4FF097536A57537A445
:106B2000124306755CA5755DB9901205E0FEA3E001
:106B3000FF900E4812D480AC83AD828C5E8D5F7561
:106B4000610475600012D265EFB4FF0DEEB4FF0969
:106B50007536A57537BD12430680097536A575379C
:106B6000D212430622222230030A9011FFE0900D38
:106B7000C4F0801C900DC4E0F539753800901210F7
:106B8000E0F53A7401F53B753CA0753DB412435AEB
:106B9000229011FEE0F8A3E0900E3BC8F0A3C8F0ED
:106BA00090123DE4F0A304F090123DE0FEA3E0FF5C
:106BB000900E3BE0FCA3E0FDEDC39FEC9E402E75E4
:106BC00039C87538001246CA90123DE0FEA3E0FFB6
:106BD0007401BE0006D39F4002801290123EE02452
:106BE00001F0500790123DE03400F050BB2230031A
:106BF00003026D3B900EDDE0F539753800753A0003
:106C00007402F53B753CA0753DB712435A900EDEF9
:106C1000E0F539753800753A007402F53B753CA013
:106C2000753DB712435A900DDBE0F53975380075A4
:106C30003A007402F53B753CA0753DB712435A907B
:106C40000DC8E0FEA3E0FF8E388F39753A0074045A
:106C5000F53B753CA5753DED12435A900EDDE09075
:106C6000123FF8E4F0E8A3F090123FE0FEA3E0FF4B
:106C7000900EDEE06F4E7003026D3B8E048F057F39
:106C800007900EDF12D414E0F539753800753A001C
:106C90007402F53B753CA0753DB712435A90123F04
:106CA000E0FEA3E0FF8E048F057F07900EE012D474
:106CB00014E0F538A3E0F539753A007402F53B7538
:106CC0003CA0753DB712435A90123FE0FEA3E0FF8F
:106CD0008E048F057F07900EE212D414E0F539750B
:106CE0003800753A007402F53B753CA0753DB7124B
:106CF000435A90123FE0FEA3E0FF8E048F057F070A
:106D0000900EE312D414AE83AF828E3E8F3F90126A
:106D100010E0F5407541A07542B412445E90123FF8
:106D2000E0FEA3E0FF0FBF00010E741F52077E00BC
:106D300090123FEEF0A3EFF0026C68223003451290
:106D40004094C006C007754C11754DFDD007D006A4
:106D50008E4E8F4F12CD53C0E0D006EE6402601C01
:106D60007535057402F5377536007401F5397538D7
:106D700000753A11753BFD12456E80067404900D46
:106D8000CCF0801A7535057400F53775360074013E
:106D9000F539753800753A10753B3212456E223060
:106DA0000345124094C006C007754C11754DFDD0C7
:106DB00007D0068E4E8F4F12CD53C0E0D006EE6442
:106DC00002601C7535057402F5377536007400F5E0
:106DD00039753800753A11753BFD12456E800674A1
:106DE00004900DCCF0801A7535057400F5377536B2
:106DF000007400F539753800753A10753B3212454C
:106E00006E2212425EC2CA7400F5CCF5CDD2CAD24F
:106E1000CF45E0900DB0F0C2CAE5CD901241F0E54B
:106E2000CC901242F0D2CA901241E0FEA3E0FF746F
:106E30000E1200038E388F39901210E0F53A74016B
:106E4000F53B753CA0753DBF12435A7536A67537A4
:106E500018124306900DB2E0FEA3E0FF8E388F3982
:106E6000901210E0F53A7401F53B753CA0753DB405
:106E700012435A223003539011FFE0900DCEF09050
:106E800011FFE060397535017400F53775360090F3
:106E90000DCEE0F539753800753A10753B32124564
:106EA0006E7400900DCDF0900DCCF07538017539F1
:106EB000F41246CA7400900DCDF0900DCCF0740021
:106EC000900DCDF0900DCCF0804F900DCAE0602D6C
:106ED0007536A07537B4124306900DCEE0F53975BE
:106EE0003800901210E0F53A7402F53B900DD1E0B5
:106EF000FEA3E0FF8E3C8F3D12435A801C900DCEC6
:106F0000E0F539753800901210E0F53A7402F53B5F
:106F1000753CA0753DB412435A2222222230030A46
:106F20009011FFE0900003F08019900003E0F53924
:106F3000753800753A017402F53B753CA0753DB497
:106F400012435A2230032F9011FFE0901270F090FC
:106F50001270E07007D3920692B28018901270E01F
:106F6000FE900003E06E6007C3920692B28005D3E4
:106F7000920692B28027A2B2B3B35006A206B3B370
:106F800040028019900003E0F539753800753A0128
:106F90007402F53B753CA0753DB412435A22300390
:106FA0002A9011FFE0901271F030B208901271E057
:106FB0009011F1F0901271E0FE9011F1E06E600717
:106FC000C3920692B28002D206801F30B21C90118A
:106FD000F1E0F539753800901210E0F53A7401F5DA
:106FE0003B753CA6753D2112435A22300356901240
:106FF00008E0FE901206E0F4042EC3940490009280
:10700000F0900092E0C3947F5032901205E0FEA30E
:10701000E0FF900E4C12D480AC83AD828C5C8D5D11
:10702000755E00755F12900092E0F5617560001268
:10703000D33D901208E0900EC9F080067404900DC4
:10704000CCF08027900092E060217536A675372439
:10705000124306753600753712900092E0F538122B
:1070600043257536A07537B4124306223003469087
:107070001208E0FE901206E0F4042EC3940490017E
:1070800013F0900113E0C3947F5022755C0E755D80
:107090004C755E00755F93900113E0F561756000BB
:1070A00012D33D901208E0900EC9F080067404904F
:1070B0000DCCF08027900113E060217536A675375E
:1070C0002A124306753600753793900113E0F538A0
:1070D0001243257536A07537B41243062230034695
:1070E000901208E0FE901206E0F4042EC39404907F
:1070F0000194F0900194E0C3947F5022755C0E756A
:107100005D4C755E01755F14900194E0F5617560EA
:107110000012D33D901208E0900EC9F0800674046E
:10712000900DCCF08027900194E060217536A67513
:107130003730124306753601753714900194E0F527
:10714000381243257536A07537B412430622300332
:1071500046901208E0FE901206E0F4042EC3940458
:10716000900215F0900215E0C3947F5022755C0EDA
:10717000755D4C755E01755F95900215E0F5617562
:10718000600012D33D901208E0900EC9F0800674A2
:1071900004900DCCF08027900215E060217536A692
:1071A000753736124306753601753795900215E02E
:1071B000F5381243257536A07537B41243062230D0
:1071C0000346901208E0FE901206E0F4042EC394E9
:1071D00004900296F0900296E0C3947F5022755C72
:1071E0000E755D4C755E02755F16900296E0F56156
:1071F00075600012D33D901208E0900EC9F0800631
:107200007404900DCCF08027900296E060217536D2
:10721000A675373C124306753602753716900296EE
:10722000E0F5381243257536A07537B412430622AF
:10723000300346901208E0FE901206E0F4042EC3DC
:107240009404900317F0900317E0C3947F502275C5
:107250005C0E755D4C755E02755F97900317E0F5E7
:107260006175600012D33D901208E0900EC9F08065
:10727000067404900DCCF08027900317E060217510
:1072800036A6753742124306753602753797900356
:1072900017E0F5381243257536A07537B41243064A
:1072A00022300346901208E0FE901206E0F4042E0D
:1072B000C39404900398F0900398E0C3947F502205
:1072C000755C0E755D4C755E03755F18900398E0F4
:1072D000F56175600012D33D901208E0900EC9F080
:1072E00080067404900DCCF08027900398E0602114
:1072F0007536A675374812430675360375371890EC
:107300000398E0F5381243257536A07537B412435B
:107310000622300346901208E0FE901206E0F404C4
:107320002EC39404900419F0900419E0C3947F5084
:1073300022755C0E755D4C755E03755F999004193E
:10734000E0F56175600012D33D901208E0900EC91F
:10735000F080067404900DCCF08027900419E06052
:10736000217536A675374E12430675360375379963
:10737000900419E0F5381243257536A07537B4121C
:10738000430622300346901208E0FE901206E0F415
:10739000042EC3940490049AF090049AE0C3947F5E
:1073A0005022755C0E755D4C755E04755F1A900415
:1073B0009AE0F56175600012D33D901208E0900EDE
:1073C000C9F080067404900DCCF0802790049AE0F8
:1073D00060217536A6753754124306753604753725
:1073E0001A90049AE0F5381243257536A07537B423
:1073F00012430622300346901208E0FE901206E087
:10740000F4042EC3940490051BF090051BE0C39474
:107410007F5022755C0E755D4C755E04755F9B90A8
:10742000051BE0F56175600012D33D901208E090F5
:107430000EC9F080067404900DCCF0802790051BD7
:10744000E060217536A675375A1243067536047505
:10745000379B90051BE0F5381243257536A075372C
:10746000B412430622300346901208E0FE90120642
:10747000E0F4042EC3940490059CF090059CE0C3B6
:10748000947F5022755C0E755D4C755E05755F1CB2
:1074900090059CE0F56175600012D33D901208E004
:1074A000900EC9F080067404900DCCF080279005F2
:1074B0009CE060217536A675376012430675360567
:1074C00075371C90059CE0F5381243257536A0757C
:1074D00037B412430622300346901208E0FE9012A1
:1074E00006E0F4042EC3940490061DF090061DE0FF
:1074F000C3947F5022755C0E755D4C755E05755F9B
:107500009D90061DE0F56175600012D33D90120854
:10751000E0900EC9F080067404900DCCF0802790A6
:10752000061DE060217536A675376612430675366E
:107530000575379D90061DE0F5381243257536A078
:107540007537B412430622300346901208E0FE90CD
:107550001206E0F4042EC3940490069EF090069E5A
:10756000E0C3947F5022755C0E755D4C755E0675A8
:107570005F1E90069EE0F56175600012D33D90128B
:1075800008E0900EC9F080067404900DCCF08027BE
:1075900090069EE060217536A675376C124306751D
:1075A000360675371E90069EE0F53812432575366F
:1075B000A07537B412430622300346901208E0FE4D
:1075C000901206E0F4042EC3940490071FF0900775
:1075D0001FE0C3947F5022755C0E755D4C755E068E
:1075E000755F9F90071FE0F56175600012D33D90B5
:1075F0001208E0900EC9F080067404900DCCF08063
:107600002790071FE060217536A675377212430672
:1076100075360675379F90071FE0F53812432575BC
:1076200036A07537B412430622300346901208E0A4
:10763000FE901206E0F4042EC394049007A0F0908C
:1076400007A0E0C3947F5022755C0E755D4C755E9B
:1076500007755F209007A0E0F56175600012D33DCB
:10766000901208E0900EC9F080067404900DCCF0E2
:1076700080279007A0E060217536A6753778124301
:10768000067536077537209007A0E0F538124325B8
:107690007536A07537B4124306223003469012089F
:1076A000E0FE901206E0F4042EC39404900821F04A
:1076B000900821E0C3947F5022755C0E755D4C7577
:1076C0005E07755FA1900821E0F56175600012D337
:1076D0003D901208E0900EC9F080067404900DCC25
:1076E000F08027900821E060217536A675377E125C
:1076F00043067536077537A1900821E0F538124327
:10770000257536A07537B412430622300346901211
:1077100008E0FE901206E0F4042EC394049008A240
:10772000F09008A2E0C3947F5022755C0E755D4C0A
:10773000755E08755F229008A2E0F5617560001221
:10774000D33D901208E0900EC9F080067404900DAD
:10775000CCF080279008A2E060217536A6753784AA
:107760001243067536087537229008A2E0F53812E4
:1077700043257536A07537B4124306223003469070
:107780001208E0FE901206E0F4042EC3940490095F
:1077900023F0900923E0C3947F5022755C0E755D41
:1077A0004C755E08755FA3900923E0F56175600074
:1077B00012D33D901208E0900EC9F0800674049038
:1077C0000DCCF08027900923E060217536A675372F
:1077D0008A1243067536087537A3900923E0F538F9
:1077E0001243257536A07537B412430622C2031220
:1077F0006FEB12706C1270DD12714E1271BF12724B
:10780000301272A11273121273F41274651274D6CC
:107810001275471275B812762912769A12770B12E2
:10782000777C12738322901208E0FE901206E0F437
:10783000042EC39404900092F0900092E0C3947FD1
:107840005020755C0E755D4C755E00755F12900082
:1078500092E0F56175600012D33D901208E0900E41
:10786000C9F022755CA6755D90755E00755F9375B5
:10787000610475600012D3127404900113F0755CFA
:10788000A6755D95755E00755F1275610475600083
:1078900012D3127404900092F0755CA6755D9A750F
:1078A0005E01755F1475610475600012D312740473
:1078B000900194F0755CA6755D9F755E01755F958E
:1078C00075610475600012D3127404900215F0758E
:1078D0005CA6755DA4755E02755F167561047560C2
:1078E0000012D3127404900296F0755CA6755DA91F
:1078F000755E02755F9775610475600012D312742E
:1079000004900317F0755CA6755DAE755E03755F38
:107910001875610475600012D3127404900398F016
:10792000755CA6755DB3755E03755F9975610475C9
:10793000600012D3127404900419F0755CA6755D92
:10794000B8755E04755F9B75610475600012D31293
:10795000740490051BF0755CA6755DBD755E0575BC
:107960005F1C75610575600012D312740590059C4B
:10797000F0755CA6755DC3755E05755F9D756105E7
:1079800075600012D312740590061DF0755CA67523
:107990005DC9755E06755F1E75610575600012D361
:1079A00012740590069EF0755CA6755DCF755E0637
:1079B000755F9F75610575600012D312740590079D
:1079C0001FF0755CA6755DD5755E07755F207561E6
:1079D0000575600012D31274059007A0F0755CA6BF
:1079E000755DDB755E07755FA175610575600012D9
:1079F000D3127405900821F0755CA6755DE1755E83
:107A000008755F2275610575600012D312740590C8
:107A100008A2F0755CA6755DE7755E08755FA375D5
:107A2000610575600012D3127405900923F0755C2E
:107A3000A6755DED755E00755F93756104756000F8
:107A400012D3127404900113F0755CA6755DF27583
:107A50005E04755F1A75610475600012D3127404B8
:107A600090049AF07432900005F8E4F0E8A3F02254
:107A7000300353901207E0FEA3E0FF901205E0FCF4
:107A8000A3E0FD12D4B074041200039010DAEEF0FB
:107A9000A3EFF07404BE00039F5023755C0E755D68
:107AA0004C755E10755FDC9010DAE0F560A3E0F5D0
:107AB0006112D33D901208E0900EC9F08006740464
:107AC000900DCCF0803E9010DAE0FEA3E0FF74044D
:107AD000BE00039F502E7536107537DC75380412C2
:107AE0004325743DF53512429C7536107537E0908C
:107AF00010DBE0C39404F5381243257536A07537C2
:107B0000B412430622300353901207E0FEA3E0FFB5
:107B1000901205E0FCA3E0FD12D4B074041200033F
:107B20009011DCEEF0A3EFF07404BE00039F50232D
:107B3000755C0E755D4C755E11755F5C9011DCE0D7
:107B4000F560A3E0F56112D33D901208E0900EC9F4
:107B5000F080067404900DCCF0803E9011DCE0FEC5
:107B6000A3E0FF7404BE00039F502E7536117537D5
:107B70005C753804124325743DF53512429C753608
:107B8000117537609011DDE0C39404F53812432578
:107B90007536A07537B412430622900DCEE09012D0
:107BA00072F07536A77537071243067536A075371C
:107BB000B41243067536D27537DE1243067536A702
:107BC00075374D124306900DCEE0F53975380075C6
:107BD0003A017402F53B900DD1E0FEA3E0FF8E3C2C
:107BE0008F3D12435A900DCAE060227536A7753753
:107BF0005E124306900000E0F539753800753A01D1
:107C00007402F53B753CA0753DB412435A900DCA01
:107C1000E0B40A028003027D069011DF7401F09047
:107C200011DFE0FE900E2BE0C39E5003027D039017
:107C300011DFE0F539753800753A017402F53B75CE
:107C40003CA0753DB712435A7535017400F5377580
:107C500036009011DFE0F539753800753A10753B44
:107C60003212456E7400900DCDF0900DCCF0753849
:107C7000017539F41246CA900DCEE060347536A70E
:107C8000753775124306900DCEE0F53975380090C2
:107C90001210E0F53A7402F53B900DD1E0FEA3E03E
:107CA000FF8E3C8F3D12435A7538017539F41246E8
:107CB000CA7535017400F5377536007400F53975ED
:107CC0003800753A10753B3212456E7538017539BA
:107CD000F41246CA7400900DCDF0900DCCF09011C6
:107CE000DFE075F00A84AFF07E00EF4E7009753664
:107CF000A07537B41243069011DFE02401F0400371
:107D0000027C1F124C867400900DCDF0900DCCF0CB
:107D10007538017539F41246CA7400900DCDF09093
:107D20000DCCF0223003239011FFE0641E60079019
:107D300011FFE0B4190280087404900DCCF08008A3
:107D40009011FFE0900DD3F0801C900DD3E0F53939
:107D5000753800901210E0F53A7402F53B753CA0BE
:107D6000753DB412435A22900E3E7401F022900EDB
:107D70003EE4F02222754C10754D3E754E11754F44
:107D8000FD12CD96D203124DA1754C10754D3E7566
:107D90004E11754FFD12CD96D203124DA1753503CC
:107DA0007400F5377536007405F539753800753A85
:107DB00010753B3212456E227536B6753706124382
:107DC00006901081E0F539753800753A017403F5B5
:107DD0003B753CA0753DB412435A7536B6753710E5
:107DE000124306900E35E0FEA3E0FF8E388F397502
:107DF0003A017403F53B753CA0753DB412435A2219
:107E0000900DCCE0603F900DCCE09011EFF012406F
:107E100094C006C007D007D0068E4C8F4D754E100B
:107E2000754F3E12CD53C0E0D006EE70181240944C
:107E3000C006C007D007D0068E4C8F4D754E10750A
:107E40004F7B12CD969011EFE0600E9011EFE06441
:107E50002A6006900DCAE07002805F901082E0B444
:107E600001349011EFE0F539753800753A0174036B
:107E7000F53B753CA0753DB712435A9011EFE09069
:107E8000B40612D424783612D49E1243067536A056
:107E90007537B41243069011EFE4F0900DCCE4F086
:107EA000900DCDE4F0754C10754D3E754E10754F2C
:107EB0007B12CD969011F47401F07400901088F04C
:107EC000901089F8E4F0E8A3F0900004E0900DCA67
:107ED000F0901082E0600302826ED2C675380175A0
:107EE00039F41246CA900003E0D394104005900084
:107EF00003E4F0900003E07007D3920692B280058D
:107F0000C3920692B2900DCAE07003027FA9753643
:107F1000A07537B41243067536A07537B412430600
:107F20007536B675371E1243067536B6753730127C
:107F30004306901082E06401600B7536B675373FDA
:107F40001243068019901082E0F539753800753AB1
:107F5000017401F53B753CA0753DB412435A75366A
:107F6000B675374312430690000AE0FEA3E0FFEF28
:107F700064397005EE6430600B7536B6753754128F
:107F80004306801C90000AE0FEA3E0FF8E388F3984
:107F9000753A017401F53B753CA0753DB412435A26
:107FA0007536B675375A1243061248389011DF7489
:107FB00001F09011DFE0D39450500E74FF12D3E41F
:107FC0009011DFE02401F050E990000AE0FEA3E008
:107FD000FFEF64397005EE6430602B900DCAE060ED
:107FE000097536B675376E12430612786390000A2B
:107FF0007430F0A37439F07401900004F0900DCA4D
:10800000F0900DCEE4F0900E21E4F0A3F0900E205D
:10801000E4F0900E24E4F0900E26E4F0900E3FE49D
:10802000F0900E40E4F0900E47E4F0901086E4F0FB
:10803000900E29E4F0900E2AE4F0900E34E4F090D3
:108040000DCAE060227536B6753795124306900E5C
:108050002BE0F539753800753A017402F53B753C33
:10806000A0753DB412435A747890000EF8E4F0E81D
:10807000A3F0900000E0900DCEF0900DCEE0FE90C9
:108080000E2BE0C39E5005900DCEE4F0900DCAE09B
:1080900060447536B67537A3124306900000E0F5CC
:1080A00039753800753A017402F53B753CA0753D91
:1080B000B412435A7536B67537B4124306900DCED6
:1080C000E0F539753800753A017402F53B753CA04E
:1080D000753DB412435A7535017400F53775360095
:1080E000900DCEE0F539753800753A10753B3212B7
:1080F000456E9011DF7401F09011DFE0D3940A50C7
:108100001F7539FA7538001246CA900DCAE060072B
:10811000742DF53512429C9011DFE02401F050D807
:108120007536A07537B4124306900DCAE0604A75E3
:1081300036B67537CB124306900DCEE0F53975385B
:1081400000753A017402F53B900DD1E0FEA3E0FF0B
:108150008E3C8F3D12435A7536B67537D912430699
:10816000900000E0F539753800753A017402F53B6E
:10817000753CA0753DB412435A90000DE0FE90107E
:1081800073E06E600990000DE0C394064002800A1F
:1081900090000DE0901073F08008901073E0900054
:1081A0000DF0A208B3500302824090108CE0B4019D
:1081B00002800302824090108CE4F090049AE0C3A5
:1081C0009480507C900DCEE06067900DCAE060090D
:1081D0007536B67537EF12430675380175392C12AE
:1081E00046CA755C04755D1A901205E0FEA3E0FFB7
:1081F000900E4812D480AC83AD828C5E8D5F90046B
:108200009AE0F56175600012D33D901205E0FEA37F
:10821000E0FF90049AE02FFF50010E901207EEF05D
:10822000A3EFF0900E4812D480743BF0900E3DE422
:10823000F0900DCAE060097536B775370412430631
:108240009010827401F0900DCAE060227536B77507
:108250003712124306901082E0F539753800753AEE
:10826000017401F53B753CA0753DB412435A900E64
:1082700020E0B40106900E24E0700302894C900DBA
:10828000CAE0B4030280030283257536A07537B4B3
:108290001243067536B7753725124306900E21E056
:1082A000FEA3E0FF8E388F39753A017401F53B75F6
:1082B0003CA0753DB712435A900E20E0F539753851
:1082C00000753A017401F53B753CA0753DB712434A
:1082D0005A90106BE0F539753800753A007401F565
:1082E0003B753CA0753DB712435A900E24E0F5391A
:1082F000753800753A007401F53B753CA0753DB7C3
:1083000012435A900E26E0F539753800753A00741C
:1083100001F53B753CA0753DB412435A7536A07506
:1083200037B4124306900E20E4F0900E24E0B4011E
:108330000280030283E9900E3EE07006900E29E071
:1083400060030283DF900E2A7401F0900DCAE06092
:10835000317407F53512429C7536B7753761124393
:10836000067536A07537B412430675360075371298
:10837000900092E0F5381243257536A07537B41297
:108380004306901205E4F0A3F0901207E4F0A3F086
:10839000755C00755D12901205E0FEA3E0FF900E83
:1083A0004812D480AC83AD828C5E8D5F900092E0E9
:1083B000F56175600012D33D901205E0FEA3E0FF69
:1083C000900092E02FFF50010E901207EEF0A3EF05
:1083D000F0900E4812D480743BF0900E3DE4F09083
:1083E0000E24E054FE900E24F0900E24E0B402021D
:1083F00080030284AF900E3EE0700D900E3DE0B41D
:108400000106900E29E060030284A5900E2A7401F3
:10841000F0900DCAE060317407F53512429C753654
:10842000B775376F1243067536A07537B412430619
:10843000753601753714900194E0F53812432575AF
:1084400036A07537B4124306901205E4F0A3F090FD
:108450001207E4F0A3F0755C01755D14901205E05D
:10846000FEA3E0FF900E4812D480AC83AD828C5EF8
:108470008D5F900194E0F56175600012D33D90121C
:1084800005E0FEA3E0FF900194E02FFF50010E9065
:108490001207EEF0A3EFF0900E4812D480743BF078
:1084A000900E3DE4F0900E24E054FD900E24F090E8
:1084B0000E24E0B404028003028575900E3EE07045
:1084C0000D900E3DE0B40106900E29E06003028598
:1084D0006B900E2A7401F0900DCAE060317407F5BC
:1084E0003512429C7536B775377D1243067536A036
:1084F0007537B4124306753601753795900215E04D
:10850000F5381243257536A07537B412430690121C
:1085100005E4F0A3F0901207E4F0A3F0755C017598
:108520005D95901205E0FEA3E0FF900E4812D48006
:10853000AC83AD828C5E8D5F900215E0F561756055
:108540000012D33D901205E0FEA3E0FF900215E07B
:108550002FFF50010E901207EEF0A3EFF0900E489F
:1085600012D480743BF0900E3DE4F0900E24E05461
:10857000FB900E24F0900E24E0B4080280030286E3
:108580003B900E3EE0700D900E3DE0B40106900E63
:1085900029E06003028631900E2A7401F0900DCA22
:1085A000E060317407F53512429C7536B775378B2C
:1085B0001243067536A07537B41243067536027538
:1085C0003716900296E0F5381243257536A07537B8
:1085D000B4124306901205E4F0A3F0901207E4F001
:1085E000A3F0755C02755D16901205E0FEA3E0FF36
:1085F000900E4812D480AC83AD828C5E8D5F900269
:1086000096E0F56175600012D33D901205E0FEA37F
:10861000E0FF900296E02FFF50010E901207EEF05F
:10862000A3EFF0900E4812D480743BF0900E3DE41E
:10863000F0900E24E054F7900E24F0900E24E0B455
:1086400010028003028701900E3EE0700D900E3DF7
:10865000E0B40106900E29E060030286F7900E2A2E
:108660007401F0900DCAE060317407F53512429C38
:108670007536B77537991243067536A07537B4123B
:108680004306753602753797900317E0F5381243A5
:10869000257536A07537B4124306901205E4F0A391
:1086A000F0901207E4F0A3F0755C02755D979012EC
:1086B00005E0FEA3E0FF900E4812D480AC83AD82AB
:1086C0008C5E8D5F900317E0F56175600012D33DFD
:1086D000901205E0FEA3E0FF900317E02FFF50018A
:1086E0000E901207EEF0A3EFF0900E4812D48074B3
:1086F0003BF0900E3DE4F0900E24E054EF900E24F9
:10870000F0900E24E0B4200280030287C7900E3E52
:10871000E0700D900E3DE0B40106900E29E060037C
:108720000287BD900E2A7401F0900DCAE06031748A
:1087300007F53512429C7536B77537A71243067593
:1087400036A07537B4124306753603753718900393
:1087500098E0F5381243257536A07537B4124306F4
:10876000901205E4F0A3F0901207E4F0A3F0755C1A
:1087700003755D18901205E0FEA3E0FF900E48120D
:10878000D480AC83AD828C5E8D5F900398E0F56100
:1087900075600012D33D901205E0FEA3E0FF900348
:1087A00098E02FFF50010E901207EEF0A3EFF0902B
:1087B0000E4812D480743BF0900E3DE4F0900E24ED
:1087C000E054DF900E24F0900E24E0B440028003C9
:1087D00002888D900E3EE0700D900E3DE0B40106D3
:1087E000900E29E06003028883900E2A7401F090B5
:1087F0000DCAE060317407F53512429C7536B775C5
:1088000037B51243067536A07537B4124306753670
:1088100003753799900419E0F5381243257536A091
:108820007537B4124306901205E4F0A3F0901207D6
:10883000E4F0A3F0755C03755D99901205E0FEA36A
:10884000E0FF900E4812D480AC83AD828C5E8D5FC9
:10885000900419E0F56175600012D33D901205E0B7
:10886000FEA3E0FF900419E02FFF50010E901207C5
:10887000EEF0A3EFF0900E4812D480743BF0900E0F
:108880003DE4F0900E24E054BF900E24F0900E24AE
:10889000E0B48002800302894C900E3EE0700D909F
:1088A0000E3DE0B40106900E29E06003028942907B
:1088B0000E2A7401F0900DCAE0602A7536B775373C
:1088C000C31243067536A07537B4124306753604D5
:1088D00075379B90051BE0F5381243257536A0755A
:1088E00037B4124306901205E4F0A3F0901207E4A7
:1088F000F0A3F0755C04755D9B901205E0FEA3E0AB
:10890000FF900E4812D480AC83AD828C5E8D5F9058
:10891000051BE0F56175600012D33D901205E0FE85
:10892000A3E0FF90051BE02FFF50010E901207EE11
:10893000F0A3EFF0900E4812D480743BF0900E3DFF
:10894000E4F0900E24E0547F900E24F0900E20E08E
:10895000B40206900E24E07003028F4D900E24E0C6
:10896000B401028003028A14900E3EE07006900E5D
:1089700029E06003028A0A900E2A7401F0900DCA61
:10898000E0602A7536B77537D11243067536A07583
:1089900037B412430675360575371C90059CE0F513
:1089A000381243257536A07537B412430690120568
:1089B000E4F0A3F0901207E4F0A3F0755C05755D98
:1089C0001C901205E0FEA3E0FF900E4812D480AC8C
:1089D00083AD828C5E8D5F90059CE0F561756000D3
:1089E00012D33D901205E0FEA3E0FF90059CE02F1E
:1089F000FF50010E901207EEF0A3EFF0900E481218
:108A0000D480743BF0900E3DE4F0900E24E054FED0
:108A1000900E24F0900E24E0B402028003028AD368
:108A2000900E3EE0700D900E3DE0B40106900E29D0
:108A3000E06003028AC9900E2A7401F0900DCAE02A
:108A4000602A7536B77537DF1243067536A075375D
:108A5000B412430675360575379D90061DE0F5384E
:108A60001243257536A07537B4124306901205E4FB
:108A7000F0A3F0901207E4F0A3F0755C05755D9D1E
:108A8000901205E0FEA3E0FF900E4812D480AC8364
:108A9000AD828C5E8D5F90061DE0F5617560001201
:108AA000D33D901205E0FEA3E0FF90061DE02FFFEE
:108AB00050010E901207EEF0A3EFF0900E4812D482
:108AC00080743BF0900E3DE4F0900E24E054FD9055
:108AD0000E24F0900E24E0B404028003028B9290E6
:108AE0000E3EE0700D900E3DE0B40106900E29E0C0
:108AF0006003028B88900E2A7401F0900DCAE0602A
:108B00002A7536B77537EE1243067536A07537B439
:108B100012430675360675371E90069EE0F538122C
:108B200043257536A07537B4124306901205E4F05C
:108B3000A3F0901207E4F0A3F0755C06755D1E903B
:108B40001205E0FEA3E0FF900E4812D480AC83AD86
:108B5000828C5E8D5F90069EE0F56175600012D399
:108B60003D901205E0FEA3E0FF90069EE02FFF502F
:108B7000010E901207EEF0A3EFF0900E4812D48091
:108B8000743BF0900E3DE4F0900E24E054FB900E08
:108B900024F0900E24E0B408028003028C51900E61
:108BA0003EE0700D900E3DE0B40106900E29E060AD
:108BB00003028C47900E2A7401F0900DCAE0602ADF
:108BC0007536B77537FD1243067536A07537B41282
:108BD000430675360675379F90071FE0F538124338
:108BE000257536A07537B4124306901205E4F0A33C
:108BF000F0901207E4F0A3F0755C06755D9F90128B
:108C000005E0FEA3E0FF900E4812D480AC83AD8255
:108C10008C5E8D5F90071FE0F56175600012D33D9B
:108C2000901205E0FEA3E0FF90071FE02FFF500128
:108C30000E901207EEF0A3EFF0900E4812D480745D
:108C40003BF0900E3DE4F0900E24E054F7900E249B
:108C5000F0900E24E0B410028003028D10900E3EBE
:108C6000E0700D900E3DE0B40106900E29E0600327
:108C7000028D06900E2A7401F0900DCAE0602A75EC
:108C800036B875370C1243067536A07537B41243E3
:108C9000067536077537209007A0E0F53812432592
:108CA0007536A07537B4124306901205E4F0A3F0B0
:108CB000901207E4F0A3F0755C07755D2090120533
:108CC000E0FEA3E0FF900E4812D480AC83AD828C0E
:108CD0005E8D5F9007A0E0F56175600012D33D9056
:108CE0001205E0FEA3E0FF9007A0E02FFF50010E69
:108CF000901207EEF0A3EFF0900E4812D480743B70
:108D0000F0900E3DE4F0900E24E054EF900E24F02D
:108D1000900E24E0B420028003028DCF900E3EE03E
:108D2000700D900E3DE0B40106900E29E060030244
:108D30008DC5900E2A7401F0900DCAE0602A753638
:108D4000B875371B1243067536A07537B412430643
:108D50007536077537A1900821E0F538124325755F
:108D600036A07537B4124306901205E4F0A3F090D4
:108D70001207E4F0A3F0755C07755DA1901205E0A1
:108D8000FEA3E0FF900E4812D480AC83AD828C5ECF
:108D90008D5F900821E0F56175600012D33D90125F
:108DA00005E0FEA3E0FF900821E02FFF50010E90A8
:108DB0001207EEF0A3EFF0900E4812D480743BF04F
:108DC000900E3DE4F0900E24E054DF900E24F090DD
:108DD0000E24E0B440028003028E8E900E3EE070BE
:108DE0000D900E3DE0B40106900E29E06003028E66
:108DF00084900E2A7401F0900DCAE0602A7536B88E
:108E000075372A1243067536A07537B412430675B6
:108E100036087537229008A2E0F5381243257536DA
:108E2000A07537B4124306901205E4F0A3F0901237
:108E300007E4F0A3F0755C08755D22901205E0FE72
:108E4000A3E0FF900E4812D480AC83AD828C5E8D7F
:108E50005F9008A2E0F56175600012D33D901205A5
:108E6000E0FEA3E0FF9008A2E02FFF50010E901259
:108E700007EEF0A3EFF0900E4812D480743BF09010
:108E80000E3DE4F0900E24E054BF900E24F0900EBE
:108E900024E0B480028003028F4D900E3EE0700DFE
:108EA000900E3DE0B40106900E29E06003028F436E
:108EB000900E2A7401F0900DCAE0602A7536B875DC
:108EC00037391243067536A07537B4124306753626
:108ED000087537A3900923E0F5381243257536A0AD
:108EE0007537B4124306901205E4F0A3F090120710
:108EF000E4F0A3F0755C08755DA3901205E0FEA395
:108F0000E0FF900E4812D480AC83AD828C5E8D5F02
:108F1000900923E0F56175600012D33D901205E0E1
:108F2000FEA3E0FF900923E02FFF50010E901207EF
:108F3000EEF0A3EFF0900E4812D480743BF0900E48
:108F40003DE4F0900E24E0547F900E24F0900E3D0E
:108F5000E0B4010280030291949011F5E070059055
:108F600011F4E4F09011F4E0B4010E9011F6E0F584
:108F70003512429C9011F4E4F09009A9E0FE9009AA
:108F8000AAE06E70030291919011F2E4F09009A9A9
:108F9000E004547F9009A9F09009A9E090092912F2
:108FA000D495E09011DEF09011DEE0B45F079010F0
:108FB0008BE4F0809890108BE0B4011F9011DEE0FC
:108FC000C3946140099011DEE0D3947A4002800B93
:108FD0009011DEE0C394209011DEF09011DEE06489
:108FE0000860079011DEE0B47F31901207E0FEA325
:108FF000E0FFEF4E602290120712D4339011F3E09D
:10900000B401157408F53512429C7420F5351242EE
:109010009C7408F53512429C0291919011DEE0B4E7
:109020000A030291919011DEE0B42E0890108BE0BB
:10903000640160028006740D9011DEF09011DEE094
:10904000B41302D2C69011DEE0B4121F901205E0F4
:10905000FEA3E0FFEF4E600D1FBFFF011E90120741
:10906000EEF0A3EFF0740D9011DEF090108BE07035
:10907000279011DEE0B42006745E9011DEF09011AE
:10908000DEE0B42E06747E9011DEF09011DEE0B4C6
:109090002C0674409011DEF09011F3E0B4010990B9
:1090A00011DEE0F53512429C901207E0FEA3E0FFCE
:1090B000900E4812D480A883A9829011DEE08883A4
:1090C0008982F00FBF00010E747F52077E0090125C
:1090D00007EEF0A3EFF09011DEE0B40D0280030282
:1090E000919190108B7401F09011F3E0B40107742A
:1090F0000AF53512429C7400900EC9F0901205F8E2
:10910000E4F0E8A3F0901205E0FEA3E0FF90120760
:10911000E0FCA3E0FDEDD39FEC9E403A900E481298
:10912000D480E0F53512489F4024901205E0FEA35C
:10913000E0FF900E4812D480FCE0FDEC900EC9E0F8
:10914000900E4812D495EDF0900EC9E004F0901204
:109150000512002680AF901205E4F0A3F0900EC92E
:10916000E0901207F8E4F0E8A3F09011F5E0B40104
:10917000069011F47401F0901207E0FEA3E0FFEFF7
:109180004E600E900E4812D480743BF0900E3DE479
:10919000F0029A41901205E0FEA3E0FF900E481203
:1091A000D480AC83AD828C5C8D5D755E10755FDCA8
:1091B00075610475600012D2A29010DAE0FCA3E0A1
:1091C000FD7404BC00039D5003D38001C392F0EFF3
:1091D00064FF7005EE64FF6003C38001D382F0502A
:1091E00060755C10755DE0901205E0FEA3E0FF90F5
:1091F0000E4812D480AC83AD828C5E8D5F9010DA05
:10920000E0FEA3E0FF74041200038E608F6112D3AE
:109210003D901205E0FEA3E0FF9010DAE0FCA3E031
:10922000FDEF2DFDEE3CFC74048C068D071200034F
:10923000901207EEF0A3EFF0900E4812D480743B2A
:10924000F0901205E0FEA3E0FF900E4812D480AC2F
:1092500083AD828C5C8D5D755E11755F5C7561049C
:1092600075600012D2A29011DCE0FCA3E0FD740452
:10927000BC00039D5003D38001C392F0EF64FF70E4
:1092800005EE64FF6003C38001D382F05060755C1B
:1092900011755D60901205E0FEA3E0FF900E48128C
:1092A000D480AC83AD828C5E8D5F9011DCE0FEA338
:1092B000E0FF74041200038E608F6112D33D9012A0
:1092C00005E0FEA3E0FF9011DCE0FCA3E0FDEF2D44
:1092D000FDEE3CFC74048C068D071200039012070F
:1092E000EEF0A3EFF0900E4812D480743BF0901291
:1092F00006E02404900EC8F0901206E0900EC9F02B
:10930000900EC9E0900E4812D495E0643B6008903E
:109310000EC9E004F080E9900EC9E0FE900EC8E0AE
:10932000D39E4009900DCC7401F0029A0FC20AC27C
:109330000B9012107401F0900EC8E0900E4812D4F9
:1093400095E0B4240D901210E4F0900EC8E004F003
:1093500080E5900EC8E0900E4812D495E0B44E0E11
:109360007402901210F0900EC8E004F080C9900EC4
:10937000C8E0900E4812D495E0B4500E74039012D9
:1093800010F0900EC8E004F080AD900EC8E0900E92
:109390004812D495E0B4490E7405901210F0900E66
:1093A000C8E004F08091900EC8E0900E4812D49569
:1093B000E0B43A0F7402901210F0900EC8E004F07E
:1093C000029337900EC8E0900E4812D495E0B42373
:1093D0000BD20B900EC8E004F0029337900EC8E059
:1093E000900E4812D495E0B42D0BD20A900EC8E02E
:1093F00004F0029337900EC8E0900E4812D495E026
:10940000B42B09900EC8E004F0029337900EC8E028
:10941000900E4812D495E0B421159011F27401F029
:109420009012107401F0900EC8E004F0029337908F
:109430000EC8E0900E4812D495E0B4261574029040
:1094400011F2F07402901210F0900EC8E004F002D5
:109450009337900EC8E0FE900EC9E06E6004D20310
:109460008002C2039011E0E4F0A3F074969011E43E
:10947000F8E4F0E8A3F09011E0E0FEA3E0FF901123
:10948000E4E0FCA3E0FDEDC39FEC9E5003029A09CB
:10949000EF2DFDEE3CFC74018C068D0712D441903B
:1094A00011E2EEF0A3EFF09011DFE4F09011DFE0B5
:1094B000D39403400302956E9011DFE0FF7E00908D
:1094C00011E2E0FCA3E0FD8E028F037F1090A778ED
:1094D00012D4148A068B0712D475E493901205FAFD
:1094E000E0FEA3E0FF9011DFE02FFF50010E900E91
:1094F0004812D480EAFEE0FFEED39F40101DBDFF6E
:10950000011C9011E4ECF0A3EDF0029A069011DF3B
:10951000E0FF7E009011E2E0FCA3E0FD8E028F03ED
:109520007F1090A77812D4148A068B0712D475E4A2
:1095300093901205FAE0FEA3E0FF9011DFE02FFF09
:1095400050010E900E4812D480EAFEE0FFEEC39F59
:1095500050100DBD00010C9011E0ECF0A3EDF002F5
:109560009A069011DFE02401F040030294ACA203BC
:10957000B3501A9011E2E0FEA3E0FF8E048F057F46
:109580001090A77E12D414E49364026002800974E0
:1095900002900DCCF0029A0F3003189011E2E0FE19
:1095A000A3E0FF8E048F057F1090A77E12D414E4F1
:1095B00093600280097409900DCCF0029A0F300379
:1095C000199011E2E0FEA3E0FF8E048F057F10905A
:1095D000A77E12D414E493B4030302986A9011E2B4
:1095E000E0FEA3E0FF8E048F057F1090A77F12D4CA
:1095F00014AE83AF828E5C8F5D755E11755FE6750C
:10960000610375600012D3129011E2E0FEA3E0FF47
:109610008E048F057F1090A78212D414AE83AF8280
:109620008E5C8F5D755E11755FE975610375600015
:1096300012D3129011E2E0FEA3E0FF8E048F057FAB
:109640001090A78512D414AE83AF828E5C8F5D75A7
:109650005E11755FEC75610375600012D312754C75
:1096600010754D3E754E11754FFD12CD96755CB857
:10967000755D48900EC8E0900E4812D495AE83AF49
:10968000828E5E8F5F75610475600012D265EFB4E3
:10969000FF16EEB4FF12754C11754DF7754E11752E
:1096A0004FFD12CD960297CC755CB8755D4C900E4F
:1096B000C8E0900E4812D495AE83AF828E5E8F5F65
:1096C00075610475600012D265EFB4FF16EEB4FF49
:1096D00012754C11754DFA754E11754FFD12CD96E0
:1096E0000297CC755CB8755D50900EC8E0900E483E
:1096F00012D495AE83AF828E5E8F5F756103756005
:109700000012D265EFB4FF16EEB4FF12754C10755F
:109710004D3E754E11754FFD12CD960297CC755C7E
:10972000B8755D53900EC8E0900E4812D495AE8384
:10973000AF828E5E8F5F75610275600012D265EF39
:10974000B4FF15EEB4FF11754C10754D44754E11F4
:10975000754FFD12CD968074755CB8755D55900E91
:10976000C8E0900E4812D495AE83AF828E5E8F5FB4
:1097700075610275600012D265EFB4FF15EEB4FF9B
:1097800011754C10754D59754E11754FFD12CD96D2
:10979000803A900EC8E0900E4812D495AE83AF8206
:1097A0008E358F367537117538FD901210E0F5390A
:1097B000900EC9E0FE900EC8E0F4042EF53A124077
:1097C000B740097404900DCCF0029A0F754C1175D6
:1097D0004DFD754E10754F3E12CD537004C2098079
:1097E00002D209754C11754DE6754E10754F3E123B
:1097F000CD5364026003C38001D3820A5009754CC3
:1098000011754DFD12CE84300B18124094C006C065
:1098100007754C11754DFDD007D0068E4E8F4F1237
:10982000CC6C754C11754DE9754E11754FFD12CD0F
:1098300053C0E0754C11754DE6754E11754FFD1214
:10984000CD53C0E0D006EE64016003C38001D39223
:10985000F0D006EEB40203D38001C372F050097455
:1098600004900DCCF0029A0F802B9011E2E0FEA341
:10987000E0FF8E048F057F1090A78512D414AE836D
:10988000AF828E5C8F5D755E11755FFD75610375CE
:10989000600012D3129011E2E0FEA3E0FF8E048F6D
:1098A000057F1090A77C12D414E493F87401939070
:1098B0001209C8F0A3C8F0300614901209E0FEA304
:1098C000E0FF7A4F7B2EEF6B7004EE6A6003029923
:1098D0007030030302996E7536B875375C12430613
:1098E0009011DF7401F09011DFE0D39495507D90DA
:1098F00011DFE07F1090A77812D404E493F53512BD
:10990000429C9011DFE07F1090A77912D404E49379
:10991000F53512429C9011DFE07F1090A77A12D4A7
:1099200004E493F53512429C9011DFE07F1090A77C
:109930007B12D404E493F53512429C9011DFE0755C
:10994000F01084AFF07E00EF4E700E7536A07537C4
:10995000B412430612425E80077420F53512429C11
:109960009011DFE02401F040030298E68000803887
:1099700020062C901209E0FEA3E0FF7C6F7D1CEF17
:109980006D7004EE6C60187C6F7D44EF6D7004EEBA
:109990006C600C7C6F7D9EEFB5050DEEB504091271
:1099A000425E90120912D3A675363075350012400A
:1099B00058C0D0753502753600124058C0D0900E90
:1099C0003EE0B40103D38001C392F0D0D082F09284
:1099D000F0D0D082F0500280CF9011E2E0FEA3E000
:1099E000FF8E048F057F1090A77812D414AE83AF3A
:1099F000828E5C8F5D755E12755F007561047560A7
:109A00000012D3128009029476900DCC7401F0906C
:109A10000EC9E004901205F8E4F0E8A3F0901205F6
:109A2000E0FEA3E0FF901207E0FCA3E0FDEFC39D82
:109A3000EE9C400D900E3D7401F0901207E4F0A3EF
:109A4000F0227400901207F8E4F0E8A3F0901205F9
:109A5000F8E4F0E8A3F0900E3D7401F09011F47476
:109A600001F09011F57401F09011F37401F0901170
:109A7000F2E4F0900E3EE4F09011F0E4F09011F07A
:109A8000E07004D2068002C206A208B340709010B3
:109A90008C7401F0743E9011F6F0754C10754D3ECB
:109AA000754E11754FF712CD96754C10754D3E756C
:109AB0004E11754FFA12CD96754C10754D3E754E80
:109AC0000D754FB412CD96755CB8755D80755E12DC
:109AD000755F0075610575600012D31290120974EC
:109AE00058F0A374CAF09010DAE4F0A3F09011DCFF
:109AF000E4F0A3F09011EFE4F09011F1E4F07E7E39
:109B00007F0022901278E4F0758E01755C20755DFF
:109B100000755E00755F0075600975612712D312CC
:109B200075A8007580FF7590FF75A0FF75B0FFC226
:109B3000C6C2AEC2C775C18175F9F075E90075C2BC
:109B40000075C30075C40075C50075C60075B70201
:109B5000D2AED2AEC2CAC2E875C902C2CF75C800C1
:109B600074FFF5CBF5CD7448F5CAF5CCD2CAC28CDA
:109B7000C2A9C28DD2B9E58954F04405F589D2A9AC
:109B8000C29CC2ACC392999298759840758780D256
:109B90009CD2BCD2ACC28EC2ABC28FC2BBC297C277
:109BA00096E589540F4420F589A280B34033900094
:109BB00010E06009900010E0C394064002800A9013
:109BC0000010E090106EF08006740390106EF0C2EA
:109BD0008E90106EE090A0C093F58BF58DD28E80A4
:109BE0004B9012767401F0901276E0D394055032C7
:109BF000859965901276E090A0C093F58BF58DD293
:109C00008E20980280FB859965E565B40D0280146D
:109C100074FF12D3E4C298C28E901276E02401F051
:109C200050C580BD901276E090106EF074009010D8
:109C30006DF0900ED6F0755CB8755D85755E10752B
:109C40005F2F75610375600012D312755CB8755D86
:109C500088755E10755F3275610375600012D312EE
:109C6000755CB8755D8B755E10755F2C75610375DD
:109C7000600012D312755CB8755D8E755E10755FED
:109C80005975610375600012D312755CB8755D91EA
:109C9000755E10755F3575610375600012D31275BE
:109CA0005CB8755D94755E10755F3875610375609D
:109CB0000012D312755CB8755D97755E10755F3BC9
:109CC00075610375600012D312755CB8755D9A7585
:109CD0005E10755F3E75610375600012D312755C8E
:109CE000B8755D9D755E10755F44756103756000A4
:109CF00012D312755CB8755DA0755E10755F4775FF
:109D0000610375600012D312755CB8755DA3755E52
:109D100010755F4A75610375600012D312755CB8E7
:109D2000755DA6755E10755F4D75610375600012F7
:109D3000D312755CB8755DA9755E10755F5375615A
:109D40000375600012D312755CB8755DAC755E105A
:109D5000755F5675610375600012D312755CB87536
:109D60005DAF755E0D755FF475610375600012D3AC
:109D700012754C10754D3E754E10754F5F12CD9695
:109D8000754C10754D3E754E0D754FC512CD9675BF
:109D90004C10754D3E754E10754F5C12CD96754C3E
:109DA00010754D3E754E0D754FC112CD96740090D5
:109DB0000EDEF0900EDDF0901276E4F0901276E078
:109DC000D394015016901276E0900DBF12D4957482
:109DD00001F0901276E02401F050E1900DDBE4F008
:109DE000754C10754D3E754E0D754FB412CD969055
:109DF0000DC8E4F0A3F090102AE4F090102BE4F0EA
:109E0000901029E4F0901072E4F0901074E4F0A344
:109E1000F0901076E4F0A3F0C204C205754C107502
:109E20004D4D754E10754F5012CD96C202300C54E8
:109E3000900DCCE4F0900DD9E4F0900DD6E4F090C4
:109E400009AAE4F09009AAE0D3947F50169009AAD9
:109E5000E090092912D495742AF09009AAE024010F
:109E6000F050E1754C10754D3E754E10754F5C12FB
:109E7000CD967EFF7FFF8E358F3612402A900DC41F
:109E8000E4F0800B7ECD7FFF8E358F3612402A7432
:109E900005900DEAF0900DCFE4F07464900DEBF0B6
:109EA000900DECF0900ED7E4F0900ED8E4F0900E08
:109EB000D9E4F090106BE0900ED4F0900EDA7401BB
:109EC000F0900E35E4F0A3F07400900E27F0900EA1
:109ED00025F0900E24F0900E20F07400900ED4F037
:109EE000900ED5F0740590000CF0901087E4F0907F
:109EF000108B7401F0900ECAE4F090108D7401F094
:109F000090108E7401F090108F7401F090092774F6
:109F100001F074009009AAF09009A9F07400900D66
:109F2000ADF8E4F0E8A3F0900DABF8E4F0E8A3F0AE
:109F3000A20C9208901277E0F535129A429010D850
:109F4000EEF0A3EFF09010D8E0F8A3E0900DE7C892
:109F5000F0A3C8F09009287401F07536A07537B4E5
:109F6000124306D206754C10754D5C754E0D754F3B
:109F7000C112CD967EFF7FFF8E358F3612402AE5C7
:109F800081900DAFF0D2AF900DCAE4F090127874CA
:109F900001F0901082E4F0901278E0B4011474FFA4
:109FA00012D3E4900DCAE060097536B87537B21265
:109FB000430690106BE0900ED4F0900DE712D3A6FC
:109FC00080F822D207754C0012CC65900DB0F07568
:109FD0004C0012CC65900DB0F0754C0012CC659021
:109FE0000DB0F075D000A207920C129B0375996515
:109FF00074FF12D3E4C20780CC02449E0244EB02F9
:10A00000455402455602455802455A02455C0245F0
:10A010005E0245600245620249D30249D50249D732
:10A020000249D9024B82024B84024BA00259AF0273
:10A0300059B10259DE0259E00260A70260A902602C
:10A04000D60260D80259BE0259C20259C60259CA84
:10A050000259CE0259D20259D60259DA0259ED02FA
:10A0600059F10259F50259F90259FD025A01025AF1
:10A0700005025A090260B60260BA0260BE0260C2FE
:10A080000260C60260CA0260CE0260D20260E502CF
:10A0900060E90260ED0260F10260F50260F90260C1
:10A0A000FD026101303132333435363738394142BF
:10A0B000434445460D0A0020002C003A002D0000C4
:10A0C00000FCF8F0E1C2000096004B00258012C0B1
:10A0D000096068A8E8696170204465766963652055
:10A0E00049442000696170204465766963652049B0
:10A0F00044202331200069617020446576696365DE
:10A100002049442023322000475049533020206406
:10A110006F5F6770692C206770695F74656D702C64
:10A1200020677069325F74656D7020677069325F97
:10A13000616374697665203D200020536574205466
:10A140007970652C2057616974200D0A000D0A0092
:10A1500057726974696E672C20494E4D4F54494FB0
:10A160004E2C204D4F56494E474657442C20757073
:10A17000646174655F6672616D652C206E65775FE2
:10A180006672616D65200D0A006E762E72657074C0
:10A190005F76616C75652C206E756D6265725F6FA0
:10A1A0006666736574206D757465645F666C61675F
:10A1B0000D0A004D6F64652C205469746C652C2069
:10A1C000436861707465722C20646D322C20646D5C
:10A1D000330D0A002C6D6F76652E0D0A002C7374FA
:10A1E0006F702E0D0A002062726F775F636D645F7F
:10A1F000626364200D0A0042434430206D7574652B
:10A200005F636D64206D757465645F666C61672063
:10A210004245464F5245206D7574652000206D6F94
:10A220006E695F636D645F626364200D0A0020667F
:10A230007373735F636D645F626364200D0A002053
:10A240006E6578745F636D645F626364200D0A00FD
:10A2500020737973745F636D645F626364200D0AB9
:10A2600000204243443020646E756D5F636D645F0F
:10A27000626364200D0A0020313D49676E6F72658C
:10A28000204261642041636B204572726F727320BB
:10A2900066726F6D206465636B2E0D0A00203D5061
:10A2A00030202438302000203D5031202439302007
:10A2B00000203D5032202441302000203D503320EA
:10A2C0002442300D0A003135203134203133203121
:10A2D00032203131203130203039203038202020D8
:10A2E00030372030362030352030342030332030A5
:10A2F00032203031203030200D0A00506F7274202F
:10A3000026205346522076616C7565733A200D0AFB
:10A310000050302050312050322050332049452009
:10A3200053434F4E2054434F4E20205432434F4E00
:10A3300020544D4F442054324D4F44204554322038
:10A3400045543232204950204950482045430D0A97
:10A35000002020002020200020202000202020009D
:10A360002020002020000020002000434D4F4420EA
:10A3700043434F4E20200D0A002020007077725F6B
:10A380006D61782C207077725F636F756E74200D2D
:10A390000A00626364302072656373200D0A002036
:10A3A0002072656373206E6F7061726D73200D0A89
:10A3B00000426567696E204572617365200D0A0071
:10A3C000457261736520436F6D706C657465200D17
:10A3D0000A0050726F6772616D6D696E67200D0AB9
:10A3E000004261642050726F6772616D2061742059
:10A3F00052414D20005361766520436F6D706C654E
:10A400007465200D0A00556E6B6E6F776E20626169
:10A41000756420726174650D0A00417661696C6132
:10A42000626C653A202033383430302C3139323088
:10A43000302C20393630302C20343830302C20204D
:10A4400032343030200D0A00203D204355525F4603
:10A4500052414D450D0A00203D2043544C5F465269
:10A46000414D450D0A00203D20434F44455F465273
:10A47000414D450D0A00203D205354445F46524152
:10A480004D450D0A00203D204E45575F4652414D37
:10A49000450D0A00203D20574F524B5F4652414D1B
:10A4A000450D0A00203D2053455249414C5F414330
:10A4B00043554D0D0A0020636870705F636D645FE3
:10A4C000626364200D0A0062636430206368646E16
:10A4D0005F636D645F626364200D0A0062636430D1
:10A4E00020636875705F636D645F626364200D0A4A
:10A4F00000626364302073656C655F636D645F62E6
:10A500006364200D0A0056432D434D20537461743B
:10A510005F636D64200D0A007061757365645F662A
:10A520006C61672000706F6C6C5F64656C61792092
:10A5300000696E697469616C697A656420000D0A4E
:10A54000007374696C5F636D6420696E206263647C
:10A5500030200D0A005430333053657420543033AA
:10A56000302064656661756C7473200D0A00543088
:10A57000363053657420543036302064656661751A
:10A580006C7473200D0A00543039305365742054B4
:10A590003039302064656661756C7473200D0A0073
:10A5A0005431323053657420543132302064656642
:10A5B00061756C7473200D0A005431383053657422
:10A5C00020543138302064656661756C7473200DD9
:10A5D0000A0053686F772074617065207061636B47
:10A5E0002064656661756C7473200D0A00203D203F
:10A5F000746F646F5F6865616420746F646F5F740B
:10A6000061696C20737461746520726573756D6522
:10A610005F616464720D0A00206F7574206F66209C
:10A62000000D0A00425430312000524C30312000DD
:10A6300042543032200042543033200042543034EF
:10A64000200042543035200042543036200042541D
:10A6500030372000494E4932200042543038200023
:10A6600042543039200042543130200042543131BC
:10A6700020004254313220004254313320004254F1
:10A68000313420004254313520004254313620000C
:10A690004E554C4C0053545550005354444E0053A7
:10A6A000544C46005354525400454E54520050529C
:10A6B0004556004E455854005245544E004E554D97
:10A6C0004231004E554D4232004E554D4233004E00
:10A6D000554D4234004E554D4235004E554D423693
:10A6E000004E554D4237004E554D4238004E554CA8
:10A6F0004C004E554C4C0035303732372028353021
:10A70000323034292020004243442056432D313634
:10A710006220436F6E74726F6C2053797374656D31
:10A720003A0D0A436F70797269676874203139385D
:10A73000362D3230303420424344204173736F63EE
:10A740002E2C20496E632E200056622D0043757218
:10A7500072656E74204465766963653A20004465CD
:10A760006661756C74206465636B5F7479706520D5
:10A7700069733A20000D0A000000000058CA00006A
:10A7800000000000000000004155445849C5010088
:10A79000000000000300000042415544656A0100CA
:10A7A000000000FFFF000000424F4F5449DD000051
:10A7B000000000000000000042524F57544F0000BC
:10A7C0000000000000000000425345547863000080
:10A7D0000000000000000000425430316FEB030025
:10A7E00000000000000000004254303270DD030021
:10A7F000000000000000000042543033714E03009E
:10A8000000000000000000004254303471BF03001B
:10A810000000000000000000425430357230030098
:10A8200000000000000000004254303672A1030016
:10A830000000000000000000425430377312030093
:10A8400000000000000000004254303873F40300A0
:10A85000000000000000000042543039746503001D
:10A8600000000000000000004254313074D60300A4
:10A870000000000000000000425431317547030021
:10A8800000000000000000004254313275B803009F
:10A89000000000000000000042543133762903001C
:10A8A000000000000000000042543134769A03009A
:10A8B000000000000000000042543135770B030017
:10A8C000000000000000000042543136777C030095
:10A8D00000000000000000004255545377ED0300D3
:10A8E000000000000000000043484150583201C001
:10A8F00000004000000000004348444E671701007C
:10A9000000000000030000004348505066ED0100C5
:10A9100000000000FF00000043485550674101005F
:10A920000000000003000000434C45525541000068
:10A930000000000000000000444542474A25010095
:10A94000000000000A0000004445434B6F44010032
:10A9500000000000FF0000004445434E6F1D010051
:10A9600000000000FF0000004449535054790100EA
:10A9700000000000FF000000444E554D576B0100E1
:10A98000000000FFFF00000044554D504A730200D4
:10A99000000000FFFF0000004543484F4AFB010054
:10A9A000000000000100000045434F464B25000019
:10A9B000000000000000000045434F4E4B2B0000FC
:10A9C000000000000000000045445444571A0000F5
:10A9D0000000000000000000454E54525670000078
:10A9E00000000000000000004552523F4C3F0100B3
:10A9F00000000000FF000000455252414BBB010027
:10AA000000000000FF000000455252464BEC0100E0
:10AA100000000000FF0000004641435449DD0000F3
:10AA20000000000000000001464657444C9A01C057
:10AA3000000040000040000046494E4C4D4501C01A
:10AA40000000400000000000464C4456573501C04D
:10AA500000004000000000004652414D4DA101C0E1
:10AA60000000400000000000465245514D600100CA
:10AA700000000000FF00000046524D5357A30100A4
:10AA8000000040000000000047444C594E01010006
:10AA9000000000FFFF000000474C49544EFB01003E
:10AAA00000000000FF000000475255506F9E01005B
:10AAB00000000000FF0000004754313054970100AF
:10AAC00000000000FF00000048454C504F2E0100E0
:10AAD00000000000000000004941503148CC010056
:10AAE000000000FFFF000000494E4932738303005D
:10AAF0000000000000000000494E49544F2F0000A4
:10AB00000000000000000000494E50545066010053
:10AB100000000000FF0000004C41424C5081030047
:10AB200000000000000000004C415354509C000005
:10AB300000000000000000004C4249546F1B01005F
:10AB400000000000020000004C454E44516000002F
:10AB500000000000000000004C495445510801006D
:10AB600000000000FF0000004C4F4F5051840100D6
:10AB700000014000000000004C4F555451070100F7
:10AB800000000000FF0000004D454E55561F00001C
:10AB900000000000000000004D49534351DC00005C
:10ABA00000000000000000004D4F443052BF01C0C3
:10ABB00000004000000000004D4F443152CF01C062
:10ABC00000004000000000004D4F444552DF0000EF
:10ABD00000000000000000004D4F4446540F0100EB
:10ABE00000000000FF0000004D4F4E49555C000082
:10ABF00000000000000000004D4F564553EF0000DC
:10AC000000000000000000004D4F5646542F010088
:10AC100000000000FF0000004D55544554B50100F0
:10AC200000000000010000004E45585455B00000DF
:10AC300000000000000000004E4F414B589501C03D
:10AC400000004000000000004E554C4C58CA000067
:10AC500000000000000000004E554D42583201C077
:10AC600000004000000000004E554D53586B01C0DD
:10AC700000004000000000004F46535458E901C056
:10AC800000004000000000004F4B4F4B567000008A
:10AC900000000000000000005041555358EA01C078
:10ACA000000040000000000050434C52599E02003A
:10ACB00000000000FF0000005045454B5A0C020008
:10ACC000000000FFFF00000050494E535A2C0000C6
:10ACD0000000000000000000504C41595C3D0100A4
:10ACE0000000400000400000504D41585F0A010044
:10ACF00000000000FF000005504F4B455CA00280A3
:10AD000000007FFFFF000000504F4C4C5CB401007E
:10AD10000000400000400000504F52545CEB000027
:10AD20000000000001000000504F57525F53010027
:10AD300000000000014000005052414D5F770200CA
:10AD400000000000FF0000005052455655DA000098
:10AD5000000000000000000050524D545F950300B9
:10AD6000000000000000000050524F4C5FB5010091
:10AD7000000040000000000050524F4D5FDF020015
:10AD8000000000FFFF000000505345546096020091
:10AD900000000000FF0000005232333267950300CC
:10ADA00000000000000000005243565461040100FE
:10ADB000000000FFFF00000052444C5961380100C0
:10ADC000000000FFFF00000052454353616901008D
:10ADD00000004000004000005245473061EA01C0D9
:10ADE000000040000000000052454731621601C0DB
:10ADF000000040000000000052454A456242000049
:10AE0000000000000000000052455054625D010047
:10AE100000000000FF0000005245544E563A00006A
:10AE200000000000000000005245574462AB01C022
:10AE30000000400000C00000524C3031706C030034
:10AE40000000000000000000524C53456356000013
:10AE500000000000000000005253554D5655000000
:10AE600000000000000000005341444463710000F2
:10AE7000000000000000000053415645644F0000F0
:10AE800000000000000000005345454B4B3202C05B
:10AE9000000040000000000053454C45676B000077
:10AEA00000000000000000005345514D6387010081
:10AEB00000000000FF0000005345515563AE000044
:10AEC0000000000000000000534C4F57660B0000CC
:10AED0000000000000000000534D505466260000A2
:10AEE00000000000000000005352434868EE0100DB
:10AEF000000000000A0000005354413268260000A0
:10AF000000000000000000005354415467B30100EA
:10AF100000000000FF0000005354444E56C90000DA
:10AF200000000000000000005354455068B40100C8
:10AF300000004000000000005354494C693A0100F1
:10AF400000004000000000005354494D698E01008C
:10AF500000000000FF00000053544C4656E400007F
:10AF6000000000000000000053544F5069B8010079
:10AF700000004000000000005354525456FF0000EF
:10AF800000000000000000005354555056AE000071
:10AF90000000000000000000535749546A280100D7
:10AFA00000000000FF0000005359535455F5000005
:10AFB000000000000000000054414C4B6B65010094
:10AFC0000000000002000001544553546B6603006A
:10AFD0000000400000000001544852446B6701002B
:10AFE000000000000100000054494D456B91020033
:10AFF000000000FFFF0000005449544C575000006F
:10B000000000000000000000544D454E5750000065
:10B010000000000000000000544F444F6BEE0100A0
:10B0200000000000FF00000054594D456E02000072
:10B030000000000020000000545950456E740100CB
:10B040000000000020000000554E49546F440100EC
:10B0500000000000FF000000555330307A700300FC
:10B060000000000000000000555330317B05030054
:10B0700000000000000000005553415665540000D8
:10B080000000000000000000564552537B9A00006B
:10B090000000000000000000565354447D2401C00D
:10B0A000000000001E00001E574149547D6700004B
:10B0B000000000000000000057454E447D6E000077
:10B0C00000000000000000005A45524F7D7500004E
:10B0D0000000000000000000FFFFFFFF58CA000052
:10B0E0000000000000000000556E6B6E6F776E2050
:10B0F0006572726F722020202020202000556E6B18
:10B100006E6F776E20636F6D6D616E6420202020FE
:10B110002000417267756D656E74205265717569A6
:10B120007265642020200042616420686578206197
:10B130007267756D656E74202020200041726775FE
:10B140006D656E742072616E6765206572726F72D4
:10B1500000556E6B6E6F776E204469736320766165
:10B160006C756520200053656E6420746F204469FF
:10B170007363206572726F722020004469736320CC
:10B180006C6964206F70656E2E20202020202000C6
:10B19000507265726F6C6C20746F6F20736D616C90
:10B1A0006C20202000417267756D656E74206E6F93
:10B1B0007420616C6C6F77656400556E657870659E
:10B1C00063746564206D6F74696F6E2E2020004E6D
:10B1D000414B2066726F6D20446973632E202020DE
:10B1E00020202000556E6B6E6F776E20446973636C
:10B1F000206572726F722020004672616D65206E4C
:10B200006F7420666F756E642E20202020004672B9
:10B21000616D6520646F6573206E6F742065786959
:10B22000737400504C522054797065206E6F7420F6
:10B23000617661696C2E20005265747279206C69A8
:10B240006D69742065786365656465640046756E34
:10B250006374696F6E2E204E6F7420417661696C45
:10B260002E00556E6578706563746564204D6F744B
:10B27000696F6E202020004672616D6520507265F6
:10B28000762E205265636F726465640042616420AB
:10B29000566964656F206F722053796E632E20208B
:10B2A000004D697373656420437574204F75742075
:10B2B0004164727373004C6F63616C204564697400
:10B2C000204572726F722E202020004E6F20456440
:10B2D00069742054797065205365742E20202000F5
:10B2E000436F6C6F72204672616D696E67204572A4
:10B2F000726F722E00544243204E6F74204163746B
:10B300006976652E20202020200054617065206918
:10B310007320456A65637465642E202020200050E8
:10B320006F776572206973206F66662E202020205B
:10B33000202020004465636B2054797065204E6F97
:10B3400074205365742E20200042616420436C6F8A
:10B35000636B20426174746572792E202000426113
:10B36000642041434B2076616C75652E202020209F
:10B370002020004E6F204164647265737320436F18
:10B3800064652E202020200053657269616C207452
:10B39000696D656F75742E2020202020004469732C
:10B3A00063204175746F20506C6179206572726FF3
:10B3B000720044697363205365617263682045724B
:10B3C00072726F722E200042616420534D505445BA
:10B3D00020436F64652E2020202020004E6F2066C1
:10B3E00072616D65206D6F74696F6E2E2020202054
:10B3F000004261642054696D6520436F64652020BC
:10B40000202020202000B0E8B0FDB112B127B13CCF
:10B41000B151B166B17BB190B1A5B1BAB1CFB1E4D0
:10B42000B1F9B20EB223B238B24DB262B277B28C79
:10B43000B2A1B2B6B2CBB2E0B2F5B0E8B0E8B0E8D3
:10B44000B30AB31FB334B0E8B0E8B0E8B0E8B0E88E
:10B45000B0E8B0E8B0E8B0E8B0E8B349B0E8B0E8C8
:10B46000B0E8B0E8B0E8B0E8B0E8B0E8B0E8B0E81C
:10B47000B0E8B0E8B0E8B0E8B0E8B0E8B0E8B0E80C
:10B48000B0E8B0E8B0E8B0E8B0E8B0E8B0E8B0E8FC
:10B49000B0E8B0E8B0E8B0E8B0E8B0E8B0E8B0E8EC
:10B4A000B0E8B0E8B0E8B0E8B0E8B0E8B0E8B0E8DC
:10B4B000B0E8B0E8B0E8B0E8B0E8B0E8B0E8B0E8CC
:10B4C000B0E8B0E8B0E8B0E8B0E8B0E8B0E8B0E8BC
:10B4D000B0E8B0E8B0E8B0E8B0E8B0E8B0E8B0E8AC
:10B4E000B0E8B0E8B0E8B0E8B0E8B0E8B0E8B0E89C
:10B4F000B0E8B0E8B0E8B0E8B0E8B0E8B0E8B0E88C
:10B50000B0E8B0E8B0E8B0E8B0E8B0E8B0E8B0E87B
:10B51000B0E8B0E8B0E8B0E8B0E8B0E8B0E8B0E86B
:10B52000B0E8B0E8B0E8B0E8B0E8B0E8B0E8B0E85B
:10B53000B0E8B0E8B0E8B0E8B0E8B0E8B0E8B0E84B
:10B54000B0E8B0E8B0E8B0E8B0E8B0E8B0E8B0E83B
:10B55000B0E8B0E8B0E8B0E8B0E8B0E8B0E8B0E82B
:10B56000B0E8B0E8B0E8B0E8B0E8B0E8B0E8B0E81B
:10B57000B0E8B0E8B0E8B0E8B0E8B0E8B0E8B0E80B
:10B58000B0E8B0E8B0E8B0E8B0E8B0E8B0E8B0E8FB
:10B59000B0E8B0E8B0E8B0E8B0E8B0E8B0E8B0E8EB
:10B5A000B0E8B0E8B0E8B0E8B0E8B0E8B0E8B0E8DB
:10B5B000B0E8B0E8B0E8B0E8B0E8B0E8B0E8B0E8CB
:10B5C000B0E8B0E8B0E8B0E8B0E8B0E8B0E8B0E8BB
:10B5D000B0E8B0E8B0E8B0E8B0E8B0E8B0E8B0E8AB
:10B5E000B0E8B0E8B0E8B0E8B0E8B0E8B0E8B0E89B
:10B5F000B0E8B35EB373B388B39DB3B2B3C7B3DC83
:10B60000B3F1B0E8B0E86469676974203D202000B8
:10B6100064696769745F73756D203D202000537401
:10B62000617274696E672075702E2E2E200D0A00CF
:10B63000696E697469616C697A6564203D200030C7
:10B640000D0A006E762E627574746F6E5F73696793
:10B65000203D20002D2D2D0D0A0020506C732073ED
:10B6600074616E642062792E2E2E200D0A002062F5
:10B670006164206E762E627574746F6E5F73696795
:10B680003A20496E697420427574746F6E732E2E61
:10B690002E200D0A00206D61785F6465636B732056
:10B6A0003D2000206E762E6465636B5F7479706553
:10B6B000203D200020536574205479706520446536
:10B6C000636B2054797065203D2000204465636BD6
:10B6D0002054797065203D20002044656661756CBA
:10B6E00074204465636B2054797065203D200049C7
:10B6F0004E493220617420706F7765722075702E0C
:10B70000200D0A00494E493220646F6E652E200DCF
:10B710000A004E4F5720696E697469616C697A65D9
:10B7200064203D200042434430206770695F6368B5
:10B73000616E67656420646F5F6770692C20677055
:10B74000695F696E2C206770695F74656D702C206D
:10B75000677069315F616374697665203D200D0A09
:10B7600000424344302042544E2031200D0A004212
:10B770004344302042544E2032200D0A00424344BC
:10B78000302042544E2033200D0A004243443020E2
:10B7900042544E2034200D0A00424344302042548B
:10B7A0004E2035200D0A00424344302042544E20A2
:10B7B00036200D0A00424344302042544E203720A8
:10B7C0000D0A00424344302042544E2038200D0AD6
:10B7D00000424344302042544E2039200D0A00429A
:10B7E0004344302042544E203130200D0A00424361
:10B7F00044302042544E203131200D0A004243444F
:10B80000302042544E203132200D0A004243443051
:10B810002042544E203133200D0A00424344302050
:10B8200042544E203134200D0A004243443020421D
:10B83000544E203135200D0A0042434430204254FA
:10B840004E203136200D0A005245473052454731CF
:10B850004F46464F4E464F524556455254686573C3
:10B8600065206172652074686520617661696C612C
:10B87000626C6520636F6D6D616E64733A0D0A00D2
:10B880002A2A2A2A0012BFCE800000C000004000F1
:10B890000020F580278D002782E0000000000001D5
:10B8A00000000200000300001E0004000008000069
:10B8B0000708466163746F7279205265736574205E
:10B8C0002830290D0A0010AF028003D38001C392F3
:10B8D0000D900DDCE0FEA3E0FFAC23AD24EE420CA6
:10B8E000EF420D900DDCECF0A3EDF0A20D92AF2233
:10B8F00010AF028003D38001C3920D900DDCE0FEF7
:10B90000A3E0FFE523F4FCE524F4FDEE520CEF5236
:10B910000D900DDCECF0A3EDF0A20D92AF22900D96
:10B92000DCE0FEA3E0FFAC23AD24EE520CEF520DA1
:10B93000ED4C6002D322C322900DDCE0FEA3E0FFB9
:10B94000AC23AD24EE520CEF520DAA23AB24EDB57F
:10B950000B06ECB50A02D322C3228523817523008E
:10B960002210AF028003D38001C3920D900927E01B
:10B97000B4010A900927E4F0852399802C900DAD3D
:10B98000E0FEA3E0FF0FBF00010E7C037DFFEE523F
:10B990000CEF520D900DADECF0A3EDF08C0E8D0F71
:10B9A0009009AB12D480E523F0A20D92AF2285243A
:10B9B00083852582E06013852483852582E0F52335
:10B9C00012B961782412D4C080E4228524838525AD
:10B9D00082E4936014852483852582E493F5231201
:10B9E000B961782412D4C080E222901298E4F0E584
:10B9F000274526700302BA78E5287038AE26AF27AF
:10BA000074108E0C8F0DFF12D4698C0E8D0F90A0C8
:10BA1000A412D480FEE493FFEE901298E090128777
:10BA200012D495EFF0AE26AF27740412D4418E26BF
:10BA30008F27803BAE26AF27740A8E0C8F0DFF1226
:10BA4000D4698C0E8D0F90A0A412D480FEE493FFD5
:10BA5000EE901298E090128712D495EFF0AE26AFD8
:10BA600027740A8E0C8F0DFF12D3F48C268D27902D
:10BA70001298E004F002B9EF901298E09012871249
:10BA8000D4957430F0E528700B901298E00454FEC1
:10BA9000901298F0901298E0C39529502690129732
:10BAA0007401F0901297E0FE901298E0F4042529BA
:10BAB000C39E400F75233012B961901297E02401A4
:10BAC000F050E0901298E06018901298E014F09016
:10BAD0001298E090128712D495E0F52312B9618094
:10BAE000E2852A24852B2512B9CB22852C54852D5D
:10BAF000557556127557A9121E6575541075553E29
:10BB0000852C56852D57121E22B4010F75232D1238
:10BB1000B9617554127555A9121F53E52E90CBD6F5
:10BB2000F82828739012A9E0F5277526007400F50F
:10BB300028752902752AA0752BBF12B9EA9012AA9E
:10BB4000E0F5277526007400F528752902752AA0EE
:10BB5000752BBF12B9EA9012ABE0F5277526007479
:10BB600000F528752902752AA0752BBF12B9EA8045
:10BB7000287554127555997556127557A9121EA835
:10BB800075241275259912B9AE800E800C800A803A
:10BB9000088006800480028000852F2485302512CD
:10BBA000B9CB227554127555AC75560E75570D12DA
:10BBB0001EA89012B4E4F09012B4E0D3940750247D
:10BBC0009012B4E09012AC12D495E0C39430FE9081
:10BBD00012B4E090127D12D495EEF09012B4E024ED
:10BBE00001F050D32210AE028003D38001C3920D26
:10BBF000AE24AF257480520F7E00EF4E605B900E36
:10BC0000DDE014541F900EDDF0900EDDE07F079014
:10BC10000EDF12D404E523F0900EDDE07F07900ED6
:10BC2000E012D404E524F0A3E525F0900EDDE07FDA
:10BC300007900EE212D404E527F085285485295593
:10BC4000900EDDE07F07900EE312D404AE83AF8246
:10BC50008E568F57121E658059900EDEE07F07903A
:10BC60000EDF12D404E523F0900EDEE07F07900E85
:10BC7000E012D404E524F0A3E525F0900EDEE07F89
:10BC800007900EE212D404E527F085285485295543
:10BC9000900EDEE07F07900EE312D404AE83AF82F5
:10BCA0008E568F57121E65900EDEE004541F900EC4
:10BCB000DEF0A20D92AE22C28C901076E526F0A3A3
:10BCC000E527F0A20E9205900DCAE0B4031B75247F
:10BCD0000075254B12B9CB75252675240012B9AE17
:10BCE0007524A07525B412B9CBE581149012B5F076
:10BCF0009012B5E0F8900DC8E6F0A308E6F0E581F3
:10BD0000C39402F58122900DB4E0FEA3E0FFAC23C2
:10BD1000AD24EF2DFDEE3CFC900DB4ECF0A3EDF066
:10BD2000E581149012B6F09012B6E0F8900DC8E6D6
:10BD3000F0A308E6F0E581C39402F58122900DC8D6
:10BD4000E0FEA3E0FFEF4E601CE581149012B7F017
:10BD50009012B7E0F8900DC8E0F608A3E0F6900D59
:10BD6000C8E4F0A3F022222222900DD17400F0A3A7
:10BD70007455F0900DCFE4F07E027F008E238F2467
:10BD800012B8C6900DCEE4F0900DDBE4F022C20FA5
:10BD90002290102AE0700C901029E0700690102B71
:10BDA000E060028003C20F22901025E0FEA3E0FFB6
:10BDB000EF4E701774F8900DCCF090102AE4F090CC
:10BDC000102BE4F0901029E4F0800690102512D496
:10BDD00033D20F22308C11300406901072E06002D2
:10BDE0008003C20F22D20F22901074E0FEA3E0FF66
:10BDF000EF4E600A901074E4F0A3F0D20F2290107E
:10BE000076E0FEA3E0FFEF4E600CD28D901076E45A
:10BE1000F0A3F0D20F22C20F22900DCAE06021756C
:10BE200024197525C412B9CBE52CF52775260074A5
:10BE300001F5287401F529752AA0752BB412B9EA09
:10BE4000E52C90CBF4F828287375260D75271CC3B4
:10BE5000920E12BCB7807C75260D7527D0C3920E4A
:10BE600012BCB7806E75260E752784C3920E12BC65
:10BE7000B7806075260F752738C3920E12BCB78045
:10BE80005275260F7527ECC3920E12BCB78044750D
:10BE900026107527A0C3920E12BCB78036752611E6
:10BEA000752754C3920E12BCB780287526127527C9
:10BEB00008C3920E12BCB7801A7526127527BCC330
:10BEC000920E12BCB7800C752613752770C3920EA4
:10BED00012BCB72212BD3D74649012CFF8E4F0E8B2
:10BEE000A3F0900DDBE090CC12F828287302C34435
:10BEF000900DCEE0B41F1B900DD17419F0A374DC2B
:10BF0000F0900DD07401F0900E34E4F0900E2C748B
:10BF100001F0740390000DF0901073F0900DCFE4D9
:10BF2000F0900DDBE4F002C344900DCAE0600975A7
:10BF3000241A75250C12B9CB752601752728C392D2
:10BF40000E12BCB7900DDBE4F002C344900DCAE0C2
:10BF5000602675241A75252912B9CB900DE2E0FEF2
:10BF6000A3E0FF8E268F277401F5287402F529754A
:10BF70002AA0752BB412B9EA900DE2E0FEA3E0FF0F
:10BF800074166F4E700C752606752714C3920E1228
:10BF9000BCB7900DE2E0FEA3E0FF74176F4E700C8B
:10BFA0007526067527C8C3920E12BCB7900DE2E045
:10BFB000FEA3E0FF74256F4E700C75260775277C75
:10BFC000C3920E12BCB7900DE2E0FEA3E0FF741C1A
:10BFD0006F4E700C752608752730C3920E12BCB7D1
:10BFE000900DE2E0FEA3E0FF74186F4E700C752612
:10BFF000087527E4C3920E12BCB7900DE2E0FEA3D1
:10C00000E0FF74196F4E700C752609752798C3925E
:10C010000E12BCB7900DE2E0FEA3E0FF741A6F4E63
:10C02000700C75260B752700C3920E12BCB7900DCD
:10C03000E2E0FEA3E0FF741B6F4E700C75260A75DC
:10C04000274CC3920E12BCB7900DE2E0FEA3E0FFB6
:10C0500074246F4E700C75260B7527B4C3920E12A4
:10C06000BCB7900DE2E0FEA3E0FF74236F4E700CAE
:10C0700075260C752768C3920E12BCB7900DE2E0CE
:10C08000FEA3E0FF74016F4E600674066F4E700CE5
:10C09000752614752724C3920E12BCB7900DE2E0EA
:10C0A000FEA3E0FF740C6F4E700C7526147527D834
:10C0B000C3920E12BCB7900DE2E0FEA3E0FF742124
:10C0C0006F4E700C75261575278CC3920E12BCB777
:10C0D000900DE2E0FEA3E0FF74206F4E700C752619
:10C0E00016752740C3920E12BCB7900DE2E0FEA376
:10C0F000E0FF74546F4E700C7526167527F4C392CA
:10C100000E12BCB7900DE2E0FEA3E0FF74376F4E55
:10C11000600302C1B7900DCAE0600975241A752545
:10C120004512B9CB7554127555C675560E755738EC
:10C13000121EA89012BAE4F09012BAE0D3940750FD
:10C14000249012BAE09012C612D495E0C39430FE47
:10C150009012BAE090127D12D495EEF09012BAE0EF
:10C160002401F050D3901283E06020901283E0907D
:10C1700012D1F09012D1E0F52C12BE199012CFE03E
:10C18000FEA3E0FF8E238F2412BD06901284E09060
:10C1900012D1F09012D1E0F52C12BE199012CFE01E
:10C1A000FEA3E0FF8E238F2412BD06752608752797
:10C1B00030C3920E12BCB7900DDBE4F002C3449082
:10C1C0000DCAE0604375241A75255512B9CB900D40
:10C1D000E0E0FEA3E0FF8E268F277401F5287402AD
:10C1E000F529752AA0752BB712B9EA900DE2E0FE89
:10C1F000A3E0FF8E268F277401F5287402F52975B8
:10C200002AA0752BB412B9EA900DE2E0FEA3E0FF7C
:10C2100074806F4E600674FF6F4E7033900DE0E0D7
:10C22000FCA3E0FD7A017B00EC520AED520BEB4AD5
:10C23000600E752600752774C3920E12BCB7800C71
:10C24000752603752744C3920E12BCB702C31C9017
:10C250000DE0E0FEA3E0FF7401520F7E00EF4E60A0
:10C260000302C302900DCAE0604375241A75257756
:10C2700012B9CB900DE0E0FEA3E0FF8E268F27746D
:10C2800001F5287402F529752AA0752BB712B9EAB1
:10C29000900DE2E0FEA3E0FF8E268F277401F528C3
:10C2A0007402F529752AA0752BB412B9EA900DE233
:10C2B000E0FEA3E0FF740A6F4E701D900DCAE060AF
:10C2C0000975241A7525A112B9CB75260175272881
:10C2D000C3920E12BCB78028900DE2E0FEA3E0FFEF
:10C2E00074156F4E700E7526017527DCC3920E1201
:10C2F000BCB7800C752605752760C3920E12BCB7BB
:10C30000801A900DE2E0FEA3E0FF74036F4E700C04
:10C31000752602752790C3920E12BCB7900DDBE410
:10C32000F08021900DDBE4F0801A900DDBE4F080CA
:10C3300013900DDBE4F0800C900DDBE4F0800590B1
:10C340000DDBE4F0227420900E2BF0C2C675F9F0DC
:10C3500075E900D2C6900DCEE0901AB812D42478B8
:10C360003112D49E783112D3AD900DB4E0FEA3E02B
:10C37000FFEF4E6008D20F900DB412D433900DCA67
:10C38000E0B4040C900DB4E0FEA3E0FFEF4E7002A9
:10C39000801C900DB4E0FEA3E0FF8E268F27740171
:10C3A000F528752906752AA0752BB412B9EA300F45
:10C3B0000302C809900EDDE0FE900EDEE06E601212
:10C3C000900DDBE0700C900DC8E0FEA3E0FFEF4E97
:10C3D000600302C7F5900EDDE07F07900EE012D4F7
:10C3E00004E0F8A3E0900DE0C8F0A3C8F0752410B5
:10C3F00075230012B91EC0D0900DE0E0FEA3E0FF4F
:10C400007402520F7E00EF4E6003D38001C392F09E
:10C41000D0D082F0500302C7F5900EDDE07F079088
:10C420000EDF12D404E0900DDBF0900EDDE07F070C
:10C43000900EE212D404E0900DE2F8E4F0E8A3F0EC
:10C44000900EDDE07F07900EE312D404AE83AF823E
:10C450008E548F5575560D7557E4121E65900EDD7E
:10C46000E004541F900EDDF0900DCFE0600302C594
:10C470004A900DCAE0B40402800302C54AE4A20F48
:10C4800033F5277526007400F528752901752AA053
:10C49000752BB912B9EA900DDBE0F527752600740B
:10C4A00000F528752902752AA0752BB912B9EA90F2
:10C4B0000DC8E0FEA3E0FF8E268F277400F52875D7
:10C4C0002904752AA0752BB912B9EA900DDCE0FE9B
:10C4D000A3E0FF8E268F277400F528752904752A9E
:10C4E000A0752BB912B9EA900DDBE0F5277526008F
:10C4F0007400F528752902752AA0752BB712B9EAC0
:10C50000900DE0E0FEA3E0FF8E268F277400F52853
:10C51000752902752AA0752BB712B9EA900DE2E0D1
:10C52000FEA3E0FF8E268F277400F528752902757B
:10C530002AA0752BB712B9EA752C0D752DE4752E4E
:10C5400000752FA07530B412BAEB900DDBE090CCE3
:10C5500030F828287302C7F3900DE3E0900DCEF079
:10C5600002C7F302C7F3900DCAE0B4014175241B62
:10C5700075253C12B9CB900DE0E0FEA3E0FF8E26BE
:10C580008F277401F528752902752AA0752BB7121B
:10C59000B9EA900DE2E0FEA3E0FF8E268F2774013A
:10C5A000F528752904752AA0752BB412B9EA02C7BB
:10C5B000F3900DCAE0604175241B75255A12B9CB62
:10C5C000900DE0E0FEA3E0FF8E268F277401F52892
:10C5D000752902752AA0752BB712B9EA900DE2E011
:10C5E000FEA3E0FF8E268F277401F52875290475B8
:10C5F0002AA0752BB412B9EA900DE0E0FEA3E0FF8B
:10C600007402520F7E00EF4E6039900DE0E0F8A307
:10C61000E0900E10C8F0A3C8F075540D7555E47580
:10C62000560E75570D121E657410F52475230012F1
:10C63000B8C6900DE2E0FEA3E0FFEF4E7005900D4E
:10C64000DBE4F0900DE0E0FEA3E0FF7401520F7E0A
:10C6500000EF4E700D7E107F008E238F2412B8C61F
:10C66000800B7E107F008E238F2412B8F0900DE097
:10C67000E0F8A3E09012BBC8F0A3C8F0900DE2E090
:10C68000F8A3E09012BDC8F0A3C8F002C7F3900D64
:10C69000E0E0FEA3E0FF7402520F7E00EF4E606503
:10C6A000900DE2E0FEA3E0FF74016F4E702A900D42
:10C6B000E0E0F8A3E0900E06C8F0A3C8F075540DB2
:10C6C0007555E475560E755700121E657420F524D5
:10C6D00075230012B8C68028900DE0E0F8A3E09022
:10C6E0000E08C8F0A3C8F075540D7555E475560EC4
:10C6F000755703121E657440F52475230012B8C6E1
:10C70000900DDBE4F002C7F3900DCAE060417524A0
:10C710001B75257812B9CB900DE0E0FEA3E0FF8EEB
:10C72000268F277401F528752902752AA0752BB765
:10C7300012B9EA900DE2E0FEA3E0FF8E268F277487
:10C7400001F528752904752AA0752BB412B9EA9051
:10C750000DE0E0FEA3E0FF7402520F7E00EF4E609A
:10C7600038900DE2E0FEA3E0FF74106F4E70289049
:10C770000DE0E0F8A3E0900E10C8F0A3C8F07554E7
:10C780000D7555E475560E75570D121E657410F52E
:10C790002475230012B8C6802C900DE2E0FEA3E0C1
:10C7A000FF74106F4E701E900DE0E0F8A3E0900E45
:10C7B00010C8F0A3C8F075541075553E75560E7527
:10C7C000570D121E65802C900DE2E0FEA3E0FFEFF6
:10C7D0004E7005900DDBE4F08019900DE2E0FEA3B1
:10C7E000E0FFEF4E7005900DDBE4F08006740990D9
:10C7F0000DDBF08000900DCEE0901AFA12D4247870
:10C800003312D49E783312D3AD900DDE12002690F1
:10C810000DDEE0FEA3E0FF74C8BE00039F50127C53
:10C82000027D008C238D2412B8F0900DDEE4F0A37D
:10C83000F090106BE4F0A2B7400A90106BE0440156
:10C8400090106BF0A2B6400A90106BE0440290107A
:10C850006BF0A2B5400A90106BE0440490106BF0AE
:10C86000A2B3400A90106BE0440890106BF0A2A6AF
:10C87000400A90106BE0441090106BF0A2A5400AA3
:10C8800090106BE0442090106BF0A2A4400A90102E
:10C890006BE0444090106BF0A2A3400A90106BE054
:10C8A000448090106BF090106CE4F0A2A2400A90CB
:10C8B000106CE0440190106CF0A2A1400A90106C42
:10C8C000E0440290106CF0A2A0400A90106CE0448A
:10C8D0000490106CF0A295400A90106CE04408900F
:10C8E000106CF0A294400A90106CE0441090106C10
:10C8F000F0A293400A90106CE0442090106CF0A2DB
:10C9000092400A90106CE0444090106CF0A291406C
:10C910000A90106CE0448090106CF0900E28E4F0C7
:10C9200090106CE0600E74029012C5F090106CE0F4
:10C93000900E28F090106BE0600E9012C57401F01C
:10C9400090106BE0900E28F0900ED4E0FE900E2830
:10C95000E06E6041900E28E0900ED4F0900E21120F
:10C960000026900DCAE0B4032C75241B7525971280
:10C97000B9CB900E21E0FEA3E0FF8E268F27740135
:10C98000F5287403F529752AA0752BB412B9EA7538
:10C99000232E12B961900E21E0FEA3E0FFEF4E704E
:10C9A0000302CB19900ED4E0FC900E28E0B50C02E7
:10C9B000800302CB12900E21120026900DCAE06077
:10C9C0000675232C12B961900E21E0FEA3E0FF90C2
:10C9D0000005E0FCA3E0FDEFC39DEE9C500302CBFD
:10C9E0000B900E21E4F0A3F09012C5E0B40206749F
:10C9F00002900E20F09012C5E0B40106900E207453
:10CA000001F0900ED4E0900E24F0900DCAE0B40333
:10CA100002800302CACA7524A07525B412B9CB7569
:10CA2000241B7525A912B9CB900E21E0FEA3E0FFCF
:10CA30008E268F277400F528752902752AA0752B7C
:10CA4000B712B9EA900E20E0F5277526007400F5BC
:10CA500028752902752AA0752BB712B9EA900E26FF
:10CA6000E0F5277526007400F528752902752AA0BF
:10CA7000752BB712B9EA900E24E0F52775260074DD
:10CA800000F528752902752AA0752BB412B9EA752C
:10CA9000241B7525E112B9CB9012C5E0F527752648
:10CAA000007400F528752902752AA0752BB712B9F4
:10CAB000EA900E28E0F5277526007400F528752900
:10CAC00002752AA0752BB412B9EA900DCAE060393C
:10CAD0009012C5E0B4010675234712B9619012C5E2
:10CAE000E0B4020675236712B961900E24E0F527C1
:10CAF0007526007400F528752902752AA0752BB4D7
:10CB000012B9EA75233E12B9618005900E20E4F057
:10CB10008007900E21E4F0A3F0900E24E06008A2BC
:10CB2000A74002D2A78007A2A7B34002C2A77554AC
:10CB30000E75554475561075573E121E22B40109E4
:10CB400075540E755544121E82901285120026905F
:10CB50001285E0FEA3E0FF74016F4E7002D2A79031
:10CB60001285E0FEA3E0FF74646F4E7002C2A790CE
:10CB70001285E0FEA3E0FFEFD39488EE9413400704
:10CB8000901285E4F0A3F075540D7555B6121F2E62
:10CB90009012BAE4F09012BAE0D394015035755473
:10CBA0000D7555B69012BAE07F03900DB912D404FA
:10CBB000AE83AF828E568F57121E22700D9012BA1E
:10CBC000E0900DBF12D4957401F09012BAE02401E8
:10CBD000F050C2C2C72202BB2402BB7102BB8B024F
:10CBE000BB8D02BB8F02BB9102BB9302BB9502BB04
:10CBF0009702BB9902BE4902BE5702BE6502BE73D0
:10CC000002BE8102BE8F02BE9D02BEAB02BEB90251
:10CC1000BEC702BEED02BEF002BF2902BF4C02C178
:10CC2000BF02C32302C32A02C33102C33802C33F77
:10CC300002C55502C55802C56302C56602C5B102E8
:10CC4000C68E02C70802C7C702C7DA02C7ED75A2BF
:10CC500020A84CA94D854E83854F828550E012FF58
:10CC6000F075A2002285A8E0854CA832854E838508
:10CC70004F82E0F8A3E0F9A3E0FA854C83854D826A
:10CC8000E0FBA3E0FCA3E02AFAEC39F9EB38854C91
:10CC900083854D82F0A3E9F0A3EAF022E4F8F9FAE3
:10CCA000AF50854C83854D82E0A3C39430F5F0509E
:10CCB0000302CD52200047940AB3500302CD52E83C
:10CCC000FCE9FDEAFEC3CA33CAC933C9C833C8C3C5
:10CCD000CA33CAC933C9C833C8CA2ECAC93DC9C8AC
:10CCE0003CC8C3CA33CAC933C9C833C8E5F0CA2A65
:10CCF000CAC93400C9C83400C8DFAD02CD43940AA4
:10CD0000E5F0400D9411404A9406B34045E5F09497
:10CD100007C3CA33CAC933C9C833C8C3CA33CAC9A7
:10CD200033C9C833C8C3CA33CAC933C9C833C8C36F
:10CD3000CA33CAC933C9C833C84AFADF0302CD436C
:10CD400002CCA8854E83854F82E8F0A3E9F0A3EAE0
:10CD5000F0C322854C83854D82E0F8A3E0F9A3E07F
:10CD6000FA854E83854F8275F000E06830E70375E1
:10CD7000F003E0C39840157018A3E0C399400D700C
:10CD800010A3E0C39A40057008740022740165F096
:10CD900022740265F022854C83854D82E0F8A3E081
:10CDA000F9A3E0FA854E83854F82E8F0A3E9F0A36A
:10CDB000EAF022854C83854D82E0F8A3E0F9A3E0F8
:10CDC000C39401FAE99400F9E89400854C83854DF9
:10CDD00082F0A3E9F0A3EAF022854E83854F82E03A
:10CDE000A3F8E0A3F9E0FA854C83854D827C987D19
:10CDF000967E8012CFDAE5532430F0A37C0F7D427B
:10CE00007E4012CFDAE5532430F0A37C017D867E8C
:10CE1000A012CFDAE5532430F0A37C007D277E10EA
:10CE200012CFDAE5532430F0A37C007D037EE812B4
:10CE3000CFDAE5532430F0A37C007D007E6412CF6E
:10CE4000DAE5532430F0A37C007D007E0A12CFDAAD
:10CE5000E5532430F0A3EA2430F0A37400F02285D7
:10CE60004C83854D82E0F8A3E0F9A3E02401FAE9C0
:10CE70003400F9E83400854C83854D82F0A3E9F055
:10CE8000A3EAF022854C83854D82E0F8A3E0F9A364
:10CE9000E0F42401FAE9F43400F9E8F43400854CB4
:10CEA00083854D82F0A3E9F0A3EAF022854E8385C5
:10CEB0004F82E0F8A3E0F9A3E0FAAB4CAC4DEA8C6A
:10CEC000F0A485F053755200755100E98CF0A4254B
:10CED00053F553E5F03552F552E5513400F551EA7A
:10CEE0008BF0A42553F553E5F03552F552E5513456
:10CEF00000F551E98BF0A42552F552E5F035518546
:10CF00004E83854F82F0A3E552F0A3E553F02285CE
:10CF10004C83854D82E0540FFBA3E0540375F00A67
:10CF2000A42BFEA3E0540FFBA3E0540775F00AA462
:10CF30002BFDA3E0540FFBA3E0540775F00AA42BCC
:10CF4000FCA3E0540FFBA3E0540375F00AA42BFAF2
:10CF5000C0E0780079007B3C12D040ECCA2ACAC9F4
:10CF60003400C9C83400C812D040EDCA2ACAC93436
:10CF700000C9C83400C87B1E12D040EECA2ACAC9F4
:10CF80003400C9C83400C8D0E002CF9AC394174017
:10CF900009C3E9948DF9E89427F8854E83854F827B
:10CFA000E8F0A3E9F0A3EAF022854E83854F82E002
:10CFB000F8A3E0F9A3E0FA854C83854D82E0FBA35A
:10CFC000E0FCA3E0C39AFAEC99F9EB98854C8385D1
:10CFD0004D82F0A3E9F0A3EAF022885189528A53E6
:10CFE000780079007A007F19C3CA9ECAC99DC9C852
:10CFF0009CC8401ED3C55333C553C55233C552C513
:10D000005133C551CA33CAC933C9C833C8DFD9027D
:10D01000D036CA2ECAC93DC9C83CC8C3C55333C5DA
:10D0200053C55233C552C55133C551CA33CAC9332A
:10D03000C9C833C8DFB2C813C8C913C9CA13CA22C2
:10D04000EA8BF0A4FAAFF0E98BF0A42FF9E5F03405
:10D0500000FFE88BF0A42FF82210AF028003D380EA
:10D0600001C39212900927E0B4010A900927E4F065
:10D07000856299802C900DADE0FEA3E0FF0FBF000C
:10D08000010E7C037DFFEE521CEF521D900DADECA6
:10D09000F0A3EDF08C1E8D1F9009AB12D480E562D9
:10D0A000F0A21292AF22856383856482E4936014B8
:10D0B000856383856482E493F56212D059786312A4
:10D0C000D4C080E222308C10B28290106FE0F58CD8
:10D0D000901070E0F58A8048D282901076E0F8A334
:10D0E000E0901074C8F0A3C8F0A205920490000D5F
:10D0F000E0901072F0901071E4F090107412D45D12
:10D10000E493FE740193FF12D4B890106FEEF0A375
:10D11000EFF090106FE0F58C901070E0F58AD28CF3
:10D12000901071E004F0901071E0FE90107412D431
:10D130005DEE12D424E493FE740193FF12D4B890F0
:10D14000106FEEF0A3EFF0EF4E7038901072E060C9
:10D1500006901072E014F0200406901072E0601F38
:10D16000901071E4F090107412D45DE493FE740199
:10D1700093FF12D4B890106FEEF0A3EFF08004C2CA
:10D180008CC28222BC000FBE0008ED8FF084FFAD80
:10D19000F022E4FEFF22BE000DEF60FE54F0606F4F
:10D1A00020E70302D23AEAC0E0EBC0E078017A005F
:10D1B00075F001EE20E710EF25E0FFEE33FE0AC523
:10D1C000F023C5F030E7F0EA5407F9096A7A007BEA
:10D1D00000600108C3EC9E40167004ED9F4010ED06
:10D1E0009FFDEC9EFCE5F0CA4ACA03F5F08005E518
:10D1F000F003F5F0C3EE13FEEF13FFD9D77908CA99
:10D20000CBCAD8D0EAFEEBFFD0E0FBD0E0FA22ECAC
:10D210008FF084FCED54F045F0C48FF084FEEDC433
:10D2200054F045F0C48FF084FDEEC4FE54F02DFFA1
:10D23000EE540F3CFEADF07C0022790078008FF0B8
:10D24000EC7E0820E70DC3CD33CD33C933C9C833D5
:10D25000C8DEF08449F9E5F08FF0BE00E6FD7C0001
:10D26000E9FFE8FE22AC5CAD5DAE5EAF5F05600538
:10D270006102D28D8D828C83E493A3AD82AC838FC7
:10D28000828E83F8E0687010A3AF82AE83D561E42C
:10D29000D560E17EFF7FFF22C3EF955FFFEE955ED5
:10D2A000FE22AC5CAD5DAE5EAF5F0560056102D293
:10D2B000C98D828C83E0A3AD82AC838F828E83F88C
:10D2C000E0687010A3AF82AE83D561E5D560E27EE1
:10D2D000FF7FFF22C3EF955FFFEE955EFE2256654E
:10D2E0007273696F6E3A20563531323231432020E5
:10D2F000446174653A205765642044656320323187
:10D300002031353A33303A30362032303035200D46
:10D310000A00AE5CAF5DAC5EAD5F0560056102D337
:10D32000368F828E83E493A3AF82AE838D828C830B
:10D33000F0A3AD82AC83D561E8D560E522AE5CAFE9
:10D340005DAC5EAD5F0560056102D3608F828E8348
:10D35000E0A3AF82AE838D828C83F0A3AD82AC83D9
:10D36000D561E9D560E622C0E0C0F0C083C082C0CC
:10D37000D075D010121D7BD0D0D082D083D0F0D009
:10D38000E032C0E0C0F0C083C082C0D075D00812C7
:10D39000C345D0D0D082D083D0F0D0E032E493F532
:10D3A000F0740193800BE0F5F0A3E0800486F008B0
:10D3B000E6C0E0C0F02200FCF8F0E1C200009600F8
:10D3C0004B00258012C0096068A8E832D3CBEF8DEE
:10D3D000F0A4F9A8F0EF8CF0A428F8EE8DF0A428C2
:10D3E000FEE9FF22600D782B02D3EE007830D8FEE4
:10D3F000D5E0F822EEC0E07E0012D184EFFDEEFC15
:10D40000D0E0FE227E0012D44FEF2582F582EE3569
:10D4100083F583227E0012D3CEEF2582F582EE358E
:10D4200083F5832225E0500205832582500205837F
:10D43000F58222A3E014F0B4FF0612D48BE014F0BE
:10D4400022048007C3CE13CECF13CFD5E0F622F847
:10D450008FF0A4FFE5F0CE88F0A42EFE22E0C0E01D
:10D46000A3E0F582D0E0F58322EEC0E07E0012D189
:10D4700084D0E0FE22EF2582F582EE3583F583220B
:10D48000E5822FF582E5833EF583220582D582026F
:10D4900015831582222582F5825002058322E493AA
:10D4A000F608740193F62275816875D000029FC357
:10D4B000C3EF9DFFEE9CFE22E4C39FFFE49EFE228D
:10D4C0000806B600021806220816B6FF0218162231
:10D4D000FFFFFFFFFFFFFFFFFFFFFFFFFFFFFFFF5C
:10D4E000FFFFFFFFFFFFFFFFFFFFFFFFFFFFFFFF4C
:10D4F000FFFFFFFFFFFFFFFFFFFFFFFFFFFFFFFF3C
:10D50000FFFFFFFFFFFFFFFFFFFFFFFFFFFFFFFF2B
:00000001FF
